:020000040800F2
:1000000000000220E98D0008C18C0008C38C0008A4
:10001000C58C0008C78C0008C98C000800000000CF
:10002000000000000000000000000000CB8C000871
:10003000CD8C000800000000CF8C0008D18C000897
:10004000398E0008398E0008398E0008398E000874
:10005000398E0008398E0008398E0008398E000864
:10006000398E0008398E0008398E0008398E000854
:10007000D58C0008398E0008398E0008E18C000804
:10008000398E0008398E0008398E0008398E000834
:10009000398E0008398E0008398E0008ED8C000872
:1000A000398E0008398E0008398E0008398E000814
:1000B000398E0008398E0008398E0008398E000804
:1000C000398E0008398E0008398E0008398E0008F4
:1000D000398E0008398E0008398E0008F58C00082A
:1000E000018D0008398E0008398E0008398E00080D
:1000F000398E0008398E0008398E0008398E0008C4
:10010000398E0008398E0008398E0008398E0008B3
:10011000398E0008398E0008298D0008398E0008B4
:10012000398E0008398E0008398E0008398E000893
:10013000398E0008398E0008398E0008398E000883
:10014000398E0008398E0008398E0008398E000873
:10015000398E0008398E0008398E0008398E000863
:10016000398E0008398E0008398E0008398E000853
:10017000398E0008398E0008398E00080000000012
:04018000398E0008AC
:1001880010B5054C237833B9044B13B10448AFF3C9
:1001980000800123237010BDDC0100200000000056
:1001A800FCBA000808B5034B1BB103490348AFF379
:1001B800008008BD00000000E0010020FCBA000833
:1001C800034613F8012B002AFBD1181A013870478F
:1001D80081F0004102E000BF83F0004330B54FEAF0
:1001E80041044FEA430594EA050F08BF90EA020F5D
:1001F8001FBF54EA000C55EA020C7FEA645C7FEAF0
:10020800655C00F0E2804FEA5454D4EB5555B8BF12
:100218006D420CDD2C4480EA020281EA030382EA83
:10022800000083EA010180EA020281EA0303362D15
:1002380088BF30BD11F0004F4FEA01314FF4801CE8
:100248004CEA113102D0404261EB410113F0004FFA
:100258004FEA03334CEA133302D0524263EB4303B1
:1002680094EA050F00F0A780A4F10104D5F1200E4F
:100278000DDB02FA0EFC22FA05F2801841F10001AA
:1002880003FA0EF2801843FA05F359410EE0A5F17E
:1002980020050EF1200E012A03FA0EFC28BF4CF0AF
:1002A800020C43FA05F3C01851EBE37101F0004565
:1002B80007D54FF0000EDCF1000C7EEB00006EEB72
:1002C8000101B1F5801F1BD3B1F5001F0CD34908FC
:1002D8005FEA30004FEA3C0C04F101044FEA445253
:1002E80012F5800F80F09A80BCF1004F08BF5FEADA
:1002F800500C50F1000041EB045141EA050130BDBA
:100308005FEA4C0C404141EB010111F4801FA4F15C
:100318000104E9D191F0000F04BF01460020B1FAB1
:1003280081F308BF2033A3F10B03B3F120020CDAE9
:100338000C3208DD02F1140CC2F10C0201FA0CF0C7
:1003480021FA02F10CE002F11402D8BFC2F1200C2C
:1003580001FA02F120FA0CFCDCBF41EA0C019040E2
:10036800E41AA2BF01EB0451294330BD6FEA04042B
:100378001F3C1CDA0C340EDC04F11404C4F1200216
:1003880020FA04F001FA02F340EA030021FA04F328
:1003980045EA030130BDC4F10C04C4F1200220FA7F
:1003A80002F001FA04F340EA0300294630BD21FABD
:1003B80004F0294630BD94F0000F83F4801306BF83
:1003C80081F480110134013D4EE77FEA645C18BF77
:1003D8007FEA655C29D094EA050F08BF90EA020F0E
:1003E80005D054EA000C04BF1946104630BD91EA06
:1003F800030F1EBF0021002030BD5FEA545C05D109
:100408004000494128BF41F0004130BD14F5800447
:100418003CBF01F5801130BD01F0004545F0FE41BB
:1004280041F470014FF0000030BD7FEA645C1ABFF0
:10043800194610467FEA655C1CBF0B46024650EA27
:10044800013406BF52EA033591EA030F41F4002153
:1004580030BD00BF90F0000F04BF0021704730B5D9
:100468004FF4806404F132044FF000054FF00001AE
:1004780050E700BF90F0000F04BF0021704730B56F
:100488004FF4806404F1320410F0004548BF404244
:100498004FF000013EE700BF42004FEAE2014FEA99
:1004A80031014FEA02701FBF12F07F4393F07F4F74
:1004B80081F06051704792F0000F14BF93F07F4FA6
:1004C800704730B54FF4607401F0004521F00041E9
:1004D80020E700BF50EA010208BF704730B54FF06F
:1004E80000050AE050EA010208BF704730B511F074
:1004F800004502D5404261EB41014FF4806404F1AC
:1005080032045FEA915C3FF4DCAE4FF003025FEA2D
:10051800DC0C18BF03325FEADC0C18BF033202EBB5
:10052800DC02C2F1200300FA03FC20FA02F001FA0F
:1005380003FE40EA0E0021FA02F11444C1E600BFAE
:1005480070B54FF0FF0C4CF4E06C1CEA11541DBF61
:100558001CEA135594EA0C0F95EA0C0F00F0DEF82C
:100568002C4481EA030621EA4C5123EA4C5350EA11
:10057800013518BF52EA033541F4801143F4801362
:1005880038D0A0FB02CE4FF00005E1FB02E506F0F3
:100598000042E0FB03E54FF00006E1FB03569CF048
:1005A800000F18BF4EF0010EA4F1FF04B6F5007F4E
:1005B80064F5407404D25FEA4E0E6D4146EB0606C0
:1005C80042EAC62141EA55514FEAC52040EA5E5049
:1005D8004FEACE2EB4F1FD0C88BFBCF5E06F1ED8F3
:1005E800BEF1004F08BF5FEA500E50F1000041EB2A
:1005F800045170BD06F0004646EA010140EA0200D7
:1006080081EA0301B4EB5C04C2BFD4EB0C0541EAF8
:10061800045170BD41F480114FF0000E013C00F30D
:10062800AB8014F1360FDEBF002001F0004170BD31
:10063800C4F10004203C35DA0C341BDC04F114044A
:10064800C4F1200500FA05F320FA04F001FA05F2D6
:1006580040EA020001F0004221F0004110EBD370A3
:1006680021FA04F642EB06015EEA430E08BF20EACF
:10067800D37070BDC4F10C04C4F1200500FA04F372
:1006880020FA05F001FA04F240EA020001F0004104
:1006980010EBD37041F100015EEA430E08BF20EA77
:1006A800D37070BDC4F1200500FA05F24EEA020EBF
:1006B80020FA04F301FA05F243EA020321FA04F0EE
:1006C80001F0004121FA04F220EA020000EBD370A5
:1006D8005EEA430E08BF20EAD37070BD94F0000FA5
:1006E8000FD101F00046400041EB010111F4801FD9
:1006F80008BF013CF7D041EA060195F0000F18BF8A
:10070800704703F00046520043EB030313F4801FC5
:1007180008BF013DF7D043EA0603704794EA0C0F7F
:100728000CEA135518BF95EA0C0F0CD050EA410695
:1007380018BF52EA4306D1D181EA030101F0004112
:100748004FF0000070BD50EA410606BF104619463A
:1007580052EA430619D094EA0C0F02D150EA013646
:1007680013D195EA0C0F05D152EA03361CBF104687
:1007780019460AD181EA030101F0004141F0FE4126
:1007880041F470014FF0000070BD41F0FE4141F4AA
:10079800780170BD70B54FF0FF0C4CF4E06C1CEAAA
:1007A80011541DBF1CEA135594EA0C0F95EA0C0F5F
:1007B80000F0A7F8A4EB050481EA030E52EA03351A
:1007C8004FEA013100F088804FEA03334FF080553B
:1007D80045EA131343EA12634FEA022245EA111568
:1007E80045EA10654FEA00260EF000419D4208BF19
:1007F800964244F1FD0404F5407402D25B084FEAC6
:100808003202B61A65EB03055B084FEA32024FF471
:1008180080104FF4002CB6EB020E75EB030E22BFCE
:10082800B61A754640EA0C005B084FEA3202B6EB8E
:10083800020E75EB030E22BFB61A754640EA5C003D
:100848005B084FEA3202B6EB020E75EB030E22BFCD
:10085800B61A754640EA9C005B084FEA3202B6EBCE
:10086800020E75EB030E22BFB61A754640EADC008D
:1008780055EA060E18D04FEA051545EA16754FEAEF
:1008880006164FEAC30343EA52734FEAC2025FEA0D
:100898001C1CC0D111F4801F0BD141EA00014FF09C
:1008A80000004FF0004CB6E711F4801F04BF01436D
:1008B8000020B4F1FD0C88BFBCF5E06F3FF6AFAE89
:1008C800B5EB030C04BFB6EB020C5FEA500C50F119
:1008D800000041EB045170BD0EF0004E4EEA11319C
:1008E80014EB5C04C2BFD4EB0C0541EA045170BDA3
:1008F80041F480114FF0000E013C90E645EA060EE7
:100908008DE60CEA135594EA0C0F08BF95EA0C0F14
:100918003FF43BAF94EA0C0F0AD150EA01347FF45C
:1009280034AF95EA0C0F7FF425AF104619462CE733
:1009380095EA0C0F06D152EA03353FF4FDAE104696
:10094800194622E750EA410618BF52EA43067FF4E7
:10095800C5AE50EA41047FF40DAF52EA43057FF477
:10096800EBAE12E74FF0FF3C06E000BF4FF0010C82
:1009780002E000BF4FF0010C4DF804CD4FEA410CE6
:100988007FEA6C5C4FEA430C18BF7FEA6C5C1BD0B3
:1009980001B050EA410C0CBF52EA430C91EA030F34
:1009A80002BF90EA020F0020704710F1000F91EA91
:1009B800030F58BF994208BF90422CBFD8176FEA5F
:1009C800E37040F0010070474FEA410C7FEA6C5C2D
:1009D80002D150EA013C07D14FEA430C7FEA6C5C34
:1009E800D6D152EA033CD3D05DF8040B704700BF60
:1009F8008446104662468C461946634600E000BFAE
:100A080001B5FFF7B7FF002848BF10F1000F01BD7F
:100A18004DF808EDFFF7F4FF0CBF012000205DF84A
:100A280008FB00BF4DF808EDFFF7EAFF34BF0120CF
:100A380000205DF808FB00BF4DF808EDFFF7E0FF68
:100A480094BF012000205DF808FB00BF4DF808EDB9
:100A5800FFF7CEFF94BF012000205DF808FB00BF20
:100A68004DF808EDFFF7C4FF34BF012000205DF802
:100A780008FB00BF4FEA410C7FEA6C5C02D150EAE8
:100A8800013C0AD14FEA430C7FEA6C5C02D152EA7E
:100A9800033C02D14FF0000070474FF0010070474F
:100AA8004FEA410212F5001215D211D56FF478738E
:100AB800B3EB625212D94FEAC12343F0004343EA31
:100AC800505311F0004F23FA02F018BF404270470C
:100AD8004FF00000704750EA013005D111F0004096
:100AE80008BF6FF0004070474FF00000704700BF2C
:100AF80080F0004002E000BF81F0004142001FBFCB
:100B08005FEA410392EA030F7FEA226C7FEA236CD3
:100B18006AD04FEA1262D2EB1363C1BFD2184140C8
:100B280048404140B8BF5B42192B88BF704710F05E
:100B3800004F40F4000020F07F4018BF404211F001
:100B4800004F41F4000121F07F4118BF494292EA69
:100B5800030F3FD0A2F1010241FA03FC10EB0C0095
:100B6800C3F1200301FA03F100F0004302D5494222
:100B780060EB4000B0F5000F13D3B0F1807F06D3CF
:100B880040084FEA310102F10102FE2A51D2B1F1C7
:100B9800004F40EBC25008BF20F0010040EA0300BC
:100BA8007047490040EB000010F4000FA2F1010269
:100BB800EDD1B0FA80FCACF1080CB2EB0C0200FAF3
:100BC8000CF0AABF00EBC25052421843BCBFD04041
:100BD8001843704792F0000F81F4000106BF80F4BB
:100BE80000000132013BB5E74FEA41037FEA226C7E
:100BF80018BF7FEA236C21D092EA030F04D092F049
:100C0800000F08BF0846704790EA010F1CBF00207C
:100C1800704712F07F4F04D1400028BF40F00040D9
:100C2800704712F100723CBF00F50000704700F0F9
:100C3800004343F0FE4040F4000070477FEA226220
:100C480016BF08467FEA23630146420206BF5FEAF1
:100C5800412390EA010F40F4800070474FF00003F1
:100C680004E000BF10F0004348BF40425FEA000CB8
:100C780008BF704743F0964301464FF000001CE060
:100C880050EA010208BF70474FF000030AE000BFB6
:100C980050EA010208BF704711F0004302D54042F4
:100CA80061EB41015FEA010C02BF84460146002066
:100CB80043F0B64308BFA3F18053A3F50003BCFA81
:100CC8008CF2083AA3EBC25310DB01FA02FC63442E
:100CD80000FA02FCC2F12002BCF1004F20FA02F235
:100CE80043EB020008BF20F00100704702F1200228
:100CF80001FA02FCC2F1200250EA4C0021FA02F289
:100D080043EB020008BF20EADC7070474FF0FF3C5D
:100D180006E000BF4FF0010C02E000BF4FF0010CED
:100D28004DF804CD4FEA40024FEA41037FEA226CB6
:100D380018BF7FEA236C11D001B052EA530C18BFD8
:100D480090EA010F58BFB2EB030088BFC81738BF3D
:100D58006FEAE17018BF40F0010070477FEA226C2B
:100D680002D15FEA402C05D17FEA236CE4D15FEA27
:100D7800412CE1D05DF8040B704700BF844608465B
:100D88006146FFE70FB5FFF7C9FF002848BF10F11C
:100D9800000F0FBD4DF808EDFFF7F4FF0CBF012061
:100DA80000205DF808FB00BF4DF808EDFFF7EAFFEB
:100DB80034BF012000205DF808FB00BF4DF808EDA6
:100DC800FFF7E0FF94BF012000205DF808FB00BF9B
:100DD8004DF808EDFFF7D2FF94BF012000205DF821
:100DE80008FB00BF4DF808EDFFF7C8FF34BF01202E
:100DF80000205DF808FB00BF42000ED2B2F1FE4FA2
:100E08000BD34FF09E03B3EB126209D44FEA0023D1
:100E180043F0004323FA02F070474FF00000704798
:100E280012F1610F01D1420202D14FF0FF30704739
:100E38004FF00000704700BF53B94AB9002908BFF6
:100E480000281CBF4FF0FF314FF0FF3000F07AB997
:100E5800ADF1080C6DE904CE00F006F8DDF804E009
:100E6800DDE9022304B070472DE9F0478C460E46B1
:100E78000446089D002B50D18A4217466CD9B2FA15
:100E880082FEBEF1000F0BD0CEF1200C01FA0EF657
:100E980020FA0CFC02FA0EF74CEA060C00FA0EF4E3
:100EA8003A0CBCFBF2F9BBB202FB19CC09FB03FA02
:100EB8004FEA144848EA0C46B2450AD9F61909F12E
:100EC800FF3180F02581B24540F22281A9F1020963
:100ED8003E44A6EB0A06B6FBF2F002FB106600FBE6
:100EE80003F3A4B244EA0644A34209D9E41900F181
:100EF800FF3280F00B81A34240F2088102383C4463
:100F08000021E41A40EA0940002D62D0002324FAA7
:100F18000EF42C606B60BDE8F0878B4207D9002D7A
:100F280055D0002185E841000846BDE8F087B3FAAE
:100F380083F1002940F08F80B34202D3824200F24D
:100F4800FC80841A66EB03060120B446002D40D0CD
:100F580085E81010BDE8F08712B90127B7FBF2F752
:100F6800B7FA87FEBEF1000F35D10121F61B4FEA13
:100F7800174C1FFA87F8B6FBFCF20CFB126608FB4D
:100F880002F0230C43EA0646B04207D9F61902F1EB
:100F9800FF3302D2B04200F2D2801A46361AB6FBAC
:100FA800FCF00CFB106608FB00F8A3B243EA064409
:100FB800A04507D9E41900F1FF3302D2A04500F299
:100FC800B9801846A4EB080440EA02409CE7294689
:100FD8002846BDE8F08707FA0EF7CEF1200326FA77
:100FE80003F24FEA174CB2FBFCF11FFA87F80CFB2F
:100FF800112206FA0EF620FA03F301FB08F933432F
:101008001E0C46EA0246B14500FA0EF409D9F61953
:1010180001F1FF3280F08C80B14540F289800239BD
:101028003E44A6EB0906B6FBFCF00CFB106200FB85
:1010380008F99EB246EA0246B14507D9F61900F109
:10104800FF3371D2B1456FD902383E44A6EB090689
:1010580040EA01418FE7C1F1200722FA07F88B40E7
:1010680048EA030326FA07F44FEA134EB4FBFEF9E5
:101078001FFA83FC0EFB19448E4020FA07F809FB7F
:101088000CFA48EA06084FEA184646EA0444A2451C
:1010980002FA01F200FA01F608D9E41809F1FF3062
:1010A80044D2A24542D9A9F102091C44A4EB0A047E
:1010B800B4FBFEF00EFB104400FB0CFC1FFA88F892
:1010C80048EA0444A44507D9E41800F1FF3E29D2B0
:1010D800A44527D902381C4440EA0940A0FB0289EC
:1010E800A4EB0C0CCC45C246CE4615D312D055B154
:1010F800B6EB0A036CEB0E0606FA07F7CB401F4364
:10110800CE402F606E600021BDE8F0871046F7E6FC
:101118008946DEE64645EAD2B8EB020A69EB030ED9
:101128000138E4E77046D7E718468FE78146BDE700
:10113800114676E702383C4444E7084606E7023A97
:101148003E442BE7704700BF38B50E4B054618786C
:101158004FF47A73B3FBF0F30B4A1068B0FBF3F06B
:1011680000F0AAF8044658B90F2D09D802462946B6
:101178004FF0FF3000F05EF8044B20461D6038BD8C
:10118800012038BD000000200800002004000020D5
:1011980008B50B4B03201A6842F400721A601A68EB
:1011A80042F480621A601A6842F480721A6000F091
:1011B8002FF80020FFF7C8FF07F080FC002008BDCB
:1011C800003C0240034A044B11681B780B4413602F
:1011D800704700BF4C04002000000020014B186835
:1011E800704700BF4C04002037B50190FFF7F6FFA9
:1011F8000546019C631C1EBF044B1B78E418FFF7CF
:10120800EDFF401BA042FAD303B030BD0000002020
:10121800074A0002D36800F4E06023F4E0631B048B
:101228001B0C43F0BF6343F400330343D3607047A0
:1012380000ED00E0174B30B5DC68C4F30224C4F1BC
:101248000703251D042B28BF0423062D4FF0010595
:1012580098BF002405FA03F303F1FF3388BF033C6A
:101268001940A14005FA04F4013C2240002842EA52
:1012780001024FEA0212A9BF00F16040064BD2B248
:1012880000F56140BBBF00F00F00D2B280F8002328
:101298001A5430BD00ED00E014ED00E0002808DB32
:1012A8000123420900F01F0003FA00F0014B43F844
:1012B8002200704700E100E00138B0F1807F0AD2D7
:1012C800F021064B064A586082F8231000200722B6
:1012D80098601A6070470120704700BF10E000E076
:1012E80000ED00E018210368DAB2103AB2FBF1F21F
:1012F80023F47F73054923F00303032A895C88BF1D
:1013080004338365C165806D704700BF18BB000852
:1013180070B50446FFF762FF0546002C71D0002324
:1013280084F834300223226884F83530136823F0B7
:101338000103136021680B68D8073BD40B68324D52
:1013480062681D40A368A0691343E26813432269D9
:10135800134362691343E26903431343226A134345
:10136800626A2B43042A01BFE56A266B35432B4387
:101378000B604B69042A23F0070343EA02030BD1ED
:10138800A26AE56A13433DB1F8B9012A2ED001D308
:10139800022A01D1EA012CD44B612046FFF7A2FFB3
:1013A8003F23E26D9340836000200123606584F849
:1013B800353070BDFFF712FF401B0528BAD920232E
:1013C8000320636584F8350070BDB0F5005F14D163
:1013D800032AE1D801A050F822F000BFFB1300084F
:1013E8009D130008FB130008F5130008B5F1C07F32
:1013F800D2D1402301206365E4E7022AF9D9032A00
:10140800C7E7012070BD00BF3F8010F070B590F8AD
:101418003440012C33D0012480F8344090F8354012
:10142800866D012C4FF000054FF0020425D180F89D
:10143800354004684565256825F480252560636086
:101448008368402B4FF03F030EBFA260A160E260AB
:10145800C26D08BFE1609340B360236843F0160390
:101468002360036C1BB1236843F0080323602368DF
:10147800002043F00103236070BD80F8345002203F
:1014880070BD90F83530022B03D0802343650120CE
:1014980070470523026880F835301368002023F070
:1014A80001031360704700000023F7B50822019379
:1014B800594B856D1F68C36D2E689A4016420446C5
:1014C8000CD001680868400708D5086820F00400B7
:1014D8000860AA60626D42F00102626501229A40CA
:1014E800164208D021684969090641BFAA60626DA1
:1014F80042F00202626504229A40164208D021682E
:101508000968880741BFAA60626D42F004026265FB
:1015180010229A40164210D02368196809070CD582
:10152800AA601A68500335D51B68190301D4236CC7
:1015380000E0A36C0BB1204698472022E16D8A4059
:10154800164238D023681868C60634D5AA6094F8BD
:101558003520052A1A6825D122F016021A605A6920
:1015680022F080025A61226C0AB9A26C1AB11A6878
:1015780022F008021A603F238B40AB60002384F8F6
:101588003430012384F83530236D0BB12046984759
:1015980003B0F0BD1A68D2055EBF1A6822F00802CF
:1015A8001A60C4E7500328D51B68190332D4636C4A
:1015B8000BB120469847636D002BE9D0636DDA07BD
:1015C80019D50523226884F83530136823F0010300
:1015D80013604FF41653B7FBF3F7019B01339F4297
:1015E800019302D31368DB07F7D4002384F834305F
:1015F800012384F83530E36CC7E71A6812F4807267
:1016080008D1196821F010011960012384F83420E9
:1016180084F83530E36BCBE70800002000232DE980
:10162800F74FD1F80080DFF8B4916A4A38FA03F42A
:1016380002D103B0BDE8F08F4FF0010E0EFA03FEA1
:1016480018EA0E0600F0B4804C6824F01007022F48
:1016580016D14FF00F0C4FEAD30A00EB8A0A03F0B9
:10166800070BDAF820504FEA8B0B0CFA0BFC25EA33
:101678000C0C0D6905FA0BF545EA0C05CAF8205063
:1016880003254FEA430A05FA0AF5ED43D0F800B0FE
:1016980004F0030C0BEA050B0CFA0AFC013F4CEAB8
:1016A8000B0C012FC0F800C011D8876807EA050B9A
:1016B800CF6807FA0AFC4CEA0B078760476827EAF5
:1016C8000E0EC4F300179F4047EA0E074760C7682D
:1016D8003D408F6807FA0AF73D43C560E50067D5C6
:1016E8004FF0000B4FF00F0ECDF804B0D9F844704E
:1016F80003F0030C47F48047C9F84470D9F84470E4
:10170800354D07F480470197019F23F0030707F140
:10171800804707F59C37D7F808A04FEA8C0C0EFADB
:101728000CFEA8422AEA0E0E44D005F58065A842B0
:1017380042D005F58065A84240D005F58065A842ED
:101748003ED005F58065A8423CD005F58065A842E5
:101758003AD005F58065A84238D005F58065A842DD
:1017680036D005F58065A84214BF0925082505FA75
:101778000CF545EA0E05BD60F743156814F4803F83
:101788000CBF3D4035431560556814F4003F0CBF4D
:101798003D4035435560956814F4801F0CBF3D40AB
:1017A80035439560D568A40254BF3D403543D560A4
:1017B80001333BE75D46DAE70125D8E70225D6E79E
:1017C8000325D4E70425D2E70525D0E70625CEE78B
:1017D8000725CCE7003C01400000024000380240E9
:1017E8000369194214BF0120002070470AB18161C2
:1017F80070470904FBE743690B4218BF090481617C
:101808007047000008B5044B5969014202D058617D
:1018180006F0E8FD08BD00BF003C01400168002259
:101828004B6913F4806310D06FF480634B612023FD
:10183800026380F83D3080F83E20036C80F83C203D
:1018480043F00403036401207047184670472DE9EC
:10185800F843044617469946C1F307488EB22568EF
:10186800B8F1010F0CBF6B69AB6936EA030314BF0B
:101878000120002008B9BDE8F8836B695A0516D520
:101888002B68202243F400732B606FF480636B6134
:101898000023236384F83D2084F83E30226C42F014
:1018A8000402226484F83C300120BDE8F8837B1CE4
:1018B800D5D0FFF793FCA0EB0900874201D3002F96
:1018C800CDD100232022236384F83D2084F83E30C4
:1018D800226C42F02002E4E770B504460D46164635
:1018E80023685B695B0701D5002070BD2046FFF7C0
:1018F80095FFA8B96A1CF3D0FFF770FC801B8542DE
:1019080001D3002DECD100232022236384F83D204D
:1019180084F83E30226C84F83C3042F02002226485
:10192800012070BD70B504460D461646206843690F
:1019380013F0400301D0002070BD4269D2060ED5D5
:101948006FF0100242612022236384F83D2084F85E
:101958003E30226C226484F83C30012070BDFFF7D1
:101968003DFC801BA84201D8002DDFD10023202296
:10197800236384F83D2084F83E30226C42F0200234
:10198800E8E72DE9F843044690461F46089EC1F350
:1019980007498DB22368B9F1010F0CBF5B699B69D8
:1019A80035EA03030CBF01230023434502D000207E
:1019B800BDE8F8837B1CEDD0FFF710FC801B874245
:1019C80001D3002FE6D100232022236384F83D2091
:1019D80084F83E30226C84F83C3042F020022264C5
:1019E8000120BDE8F88370B504460D461646236805
:1019F8005B691B0601D5002070BD2046FFF70EFF6E
:101A0800A8B96A1CF3D0FFF7E9FB801B854201D314
:101A1800002DECD100232022236384F83D2084F894
:101A28003E30226C84F83C3042F0200222640120CF
:101A380070BD00002DE9FF411546026898461368FD
:101A48000B9E43F4807313600F4600960A9B002296
:101A58004FF001110446FFF794FF18B1012004B0BC
:101A6800BDE8F081236807F0FE071F610A9A334634
:101A780016492046FFF7EBFE0028EFD123680390B4
:101A88005A690A9903929B69324603932046039B3D
:101A9800FFF7A9FF40B1236C042B01BF226813682C
:101AA80043F400731360D9E7B8F1010F236802D13A
:101AB800EDB21D61D3E72A0A1A610A993246204617
:101AC800FFF791FF0028E6D12368F1E70200010043
:101AD8002DE9FF419846036816461A680B9D42F4A3
:101AE80080621A601A680F4642F480721A604FF0DA
:101AF800011100950A9B00220446FFF742FF18B126
:101B0800012004B0BDE8F0812368FFB207F0FE02AF
:101B18001A6129492B460A9A2046FFF798FE0028A1
:101B2800EED1236803905A690A9903929B692A4661
:101B380003932046039BFFF756FF40B1236C042B09
:101B480001BF2268136843F400731360D8E7B8F143
:101B5800010F236825D1F6B21E612A460A9920464C
:101B6800FFF741FF02460028E8D1216820460B68AC
:101B780043F480730B6000950A9B4FF00111FFF747
:101B880000FF0028BCD1236847F001071F610A9AAB
:101B98002B4609492046FFF75AFE003018BF01209E
:101BA800AFE7320A1A610A992A462046FFF71BFF57
:101BB8000028C3D12368CEE70200010070B50446AF
:101BC80008B9012070BD90F83D3003F0FF021BB941
:101BD80080F83C2006F08EFF2423226884F83D30EC
:101BE800136823F00103136000F098FC6568414B0B
:101BF8009D424DD8404B9842E3D940492268B0FBFA
:101C0800F1F1536823F03F030B435360136A23F049
:101C18003F03013119431162D169364B21F44F4119
:101C28009D4221F0FF0100F1FF3048D86D00B0FB64
:101C3800F5F00130C0F30B03042B38BF04230B432A
:101C4800D3611168206AE36921F0C00103430B43A3
:101C580013609168E068236921F40341034321F08C
:101C6800FF010B439360D168A069636921F0FF010C
:101C780003430B43D3601368002043F00103136050
:101C88002023206484F83D30206384F83E0070BD32
:101C98001B4B984295D9194E4FF49671B0FBF6F646
:101CA80022687143536823F03F0333434FF47A7635
:101CB8005360136AB1FBF6F123F03F03A9E7A36869
:101CC80053B905EB4503B0FBF3F0431CC3F30B0317
:101CD8006BB143F40043B2E719236B43B0FBF3F055
:101CE800431CC3F30B0313B143F44043A7E7012399
:101CF800A5E700BFA08601007F841E0040420F00B8
:101D0800FF083D002DE9F743044699460F469046E3
:101D18000C9EFFF763FA94F83D300546202B03D05C
:101D2800022003B0BDE8F0830090192301223B494B
:101D38002046FFF726FE0028F2D194F83C30012B0C
:101D4800EED0012384F83C30236820461A68D10776
:101D580058BF1A6839465CBF42F001021A601A6817
:101D680022F400621A60212384F83D30402384F86D
:101D78003E30002323640A9B01956362BDF82C3032
:101D880000966385638D42462385254BE3624B4667
:101D9800FFF750FE00282AD00120C2E7FFF723FEF4
:101DA80040B1236C042B01BF2268136843F400730D
:101DB8001360F1E7636A27681A4612F8011B396154
:101DC8006262628D218D013A92B262857A69481EFB
:101DD80080B2520720850AD548B15A7802333A6151
:101DE8006362638D0239013B9BB221856385238D34
:101DF8002A4631462046002BD0D1FFF76DFD00283A
:101E0800CFD12268136843F400731360202384F849
:101E18003C0084F83D3084F83E0082E70200100060
:101E28000000FFFF2DE9F043044687B099460D46B0
:101E38009046109FFFF7D2F994F83D300646202BC4
:101E480004D00225284607B0BDE8F0830090192386
:101E5800012277492046FFF794FD0028F1D194F834
:101E68003C30012BEDD0012384F83C30236829460F
:101E78001A68D00758BF1A6820465CBF42F00102B2
:101E88001A601A6822F400621A60222384F83D302E
:101E9800402384F83E30002323640E9B019663623E
:101EA800BDF83C3000976385638D42462385614BBE
:101EB800E3624B46FFF70CFE054608B10125C1E772
:101EC800228D236892B902905A6902929A69029205
:101ED800029A1A6842F400721A60202384F83D308E
:101EE800002384F83E3084F83C30ABE7012A2CD13B
:101EF8001A6822F480621A6003905A6903929A69F8
:101F08000392039A1A6842F400721A60DFF8288173
:101F1800238D002BE1D0032B6ED8012B2DD1324617
:101F280039462046FFF7FEFC0028C7D12268636ABD
:101F380012691A70636A01336362238D013B23853A
:101F4800638D013B9BB26385E2E7022A0ED11A68D2
:101F580022F480621A601A6842F400621A600490DF
:101F68005A6904929B690493049BCFE705905A69C8
:101F780005929B690593059BC8E7022B00963B4693
:101F88004FF000024146204619D1FFF7FAFC00281D
:101F980094D123681A6842F400721A601B69626A55
:101FA8001370626A531C6362238D013B2385638D22
:101FB800013B9BB2638523681B695370BAE7FFF73F
:101FC800E0FC024600287FF479AF236820461968B0
:101FD80021F4806119601B69616A0B70636A00965D
:101FE80001336362238D4146013B2385638D013BA9
:101FF8009BB263853B46C8E7324639462046FFF721
:1020080091FC00287FF45AAF2268636A12691A703B
:10201800626A531C6362238D013B2385638D013BF8
:102028009BB263852368596949077FF571AFC3E798
:10203800020010000000FFFF040001002DE9F34139
:10204800044608B901203BE00368DD0710D4236883
:10205800980745D423681A0700F1918023685B0725
:1020680000F1AF80A069002840F00181002027E03E
:10207800AA4B9A6802F00C02042A07D09A6802F068
:102088000C02082A0AD15B68590207D5A34B1B68C2
:102098009A03DCD56368002BD9D1D3E7A04B22790A
:1020A8001A7063687BB1FFF799F806469B4D2B6859
:1020B8009B03CCD4FFF792F8801B6428F7D9032040
:1020C80002B0BDE8F081FFF789F80646934D2B680A
:1020D8009F03BCD5FFF782F8801B6428F7D9EEE789
:1020E8008E4B9A6812F00C0F07D09A6802F00C0217
:1020F800082A16D15B685E0213D4884B1A689507C4
:1021080002D5E268012A9DD11868F82292FAA2F253
:10211800B2FA82F122698A4020F0F8010A431A6073
:1021280098E7E2687F4BDAB101221A60FFF756F8A8
:1021380006467A4D2B6898070CD52968F82393FA38
:10214800A3F3B3FA83F22369934021F0F80213430F
:102158002B607FE7FFF742F8801B0228EAD9AEE739
:102168001A60FFF73BF806466C4D2B6899077FF518
:1021780071AFFFF733F8801B0228F6D99FE7626931
:10218800694B7AB101221A60FFF728F80646634DB9
:102198006B6F9F073FF562AFFFF720F8801B02289F
:1021A800F6D98CE71A60FFF719F806465B4D6B6F96
:1021B80098077FF553AFFFF711F8801B0228F6D96F
:1021C8007DE7564B1A6C12F0805226D101260192F7
:1021D8001A6C42F080521A641B6C03F0805301930E
:1021E800019B524D2B6843F480732B602B68D905F3
:1021F80015D54F4B227A1A70A36803BBFEF7EEFF82
:1022080041F288380746454D2B6F980720D5FEF7D1
:10221800E5FFC01B4045F7D951E70026E1E72B68E9
:1022280043F480732B60FEF7D9FF07462B68DA0565
:10223800DFD4FEF7D3FFC01B0228F7D93FE7FEF72C
:10224800CDFF41F288380746344D2B6F9B0708D5E0
:10225800002E3FF407AF314A136C23F08053136408
:1022680000E7FEF7BBFFC01B4045EED927E72B4D23
:10227800AB6803F00C03082B5ED000232D4E022818
:1022880033603ED1FEF7AAFF07462B68990132D486
:1022980047F6C07797FAA7F74FF44032B7FA87F7AF
:1022A80092FAA2F24FF07061B2FA82F091FAA1F1BB
:1022B800B1FA81F1226AE3691343626A02FA07F705
:1022C800A26A3B435208013A82401343E26A134C24
:1022D80002FA01F10B436B6001233360FEF77EFFC6
:1022E800054623689A013FF5C1AEFEF777FF401B0C
:1022F8006428F6D9E3E6FEF771FFC01B6428C4D949
:10230800DDE6FEF76BFF04462B689B017FF5AEAE5A
:10231800FEF764FF001B6428F6D9D0E600380240B7
:102328000238024000004742800E474200700040D9
:10233800703802406000474201283FF4C1AE686827
:10234800E36900F480029A427FF47CAE226A00F0CE
:102358003F0393427FF476AE626AC0F388139342D8
:102368007FF470AEA26A00F4403393427FF46AAE01
:10237800E36A00F07060C01A18BF0120A0E600BF31
:10238800134908B58B6803F00C03042B03D0082B02
:1023980003D0104808BD104808BD4A684B68496812
:1023A80013F4800314BF0C480A48C1F3881118BFFE
:1023B800002302F03F02A1FB0001FEF73DFD044BA4
:1023C8005B68C3F3014301335B00B0FBF3F008BD66
:1023D800003802400024F40040787D012DE9F041E6
:1023E8000D46044610B90120BDE8F081464B1A6835
:1023F80002F00F028A422FD321688F0734D4C8070E
:1024080047D4414B1A6802F00F0295426BD32268F9
:10241800510771D4130707D53C4A2169936823F4FF
:10242800604343EAC1039360FFF7AAFF374BF022EA
:102438009B6892FAA2F2B2FA82F203F0F003D34058
:10244800334AD35CD840334B1860334B1868FEF7D7
:102458007BFE0020BDE8F081CAB21A701B6803F049
:102468000F039942BFD1C7E7284B11F0040F1EBFD5
:102478009A6842F4E0529A600E0742BF9A6842F4A2
:1024880060429A609A68A06822F0F00202439A605B
:10249800B5E761681D4B01291A681CD112F4003F89
:1024A800A1D09A6841F2883822F003020A439A6060
:1024B800FEF794FE0746154EB368626803F00C03F6
:1024C800B3EB820F9DD0FEF789FEC01B4045F3D9C0
:1024D8000320BDE8F081022902D112F0007FDFE776
:1024E80012F0020FDCE7EAB21A701B6803F00F0360
:1024F8009D427FF478AF8AE70449E0688B6823F44B
:10250800E05303438B6085E7003C024000380240FB
:10251800B6BC00080800002004000020084B4FF457
:10252800E0529B6892FAA2F2B2FA82F203F4E05304
:10253800D340044AD35C044A1068D840704700BFAF
:1025480000380240C6BC000808000020084B4FF4C1
:1025580060429B6892FAA2F2B2FA82F203F46043F4
:10256800D340044AD35C044A1068D840704700BF7F
:1025780000380240C6BC000808000020036800209C
:10258800DA6842F00102DA609A6802F00702062A65
:102598001EBF1A6842F001021A6070477047704700
:1025A80070477047036810B51A69044691070ED53D
:1025B800DA6892070BD56FF002021A6101229B6953
:1025C80002779B0777D0FFF7EAFF0023237723687A
:1025D8001A69500710D5DA6851070DD56FF0040253
:1025E8001A6102229B69227713F4407F204668D043
:1025F800FFF7D5FF0023237723681A6912070FD541
:10260800DA6810070CD56FF008021A610422DB693A
:102618002277990720465AD0FFF7C1FF0023237776
:1026280023681A69D20610D5DA68D0060DD56FF07E
:1026380010021A610822DB69227713F4407F2046D2
:102648004BD0FFF7ACFF0023237723681A69D10723
:1026580008D5DA68D20705D56FF0010220461A615D
:1026680005F072FE23681A69100608D5DA681106A3
:1026780005D56FF0800220461A6100F0D4F823686F
:102688001A69520608D5DA68500605D56FF0400277
:1026980020461A61FFF785FF23681A69910622D53B
:1026A800DA6892061FD56FF020022046BDE8104078
:1026B8001A6100F0B7B8FFF771FF2046FFF770FF07
:1026C80083E7FFF76BFF2046FFF76AFF92E7FFF704
:1026D80065FF2046FFF764FFA0E7FFF75FFF20468E
:1026E800FFF75EFFAFE710BD304A0368904212D093
:1026F800B0F1804F0FD0A2F57C4290420BD002F58A
:102708008062904207D002F58062904203D002F5C1
:102718007842904219D14A6823F070031343234A40
:10272800904229D0B0F1804F26D0A2F57C42904249
:1027380022D002F5806290421ED002F5806290425B
:102748001AD002F57842904216D0194A904213D016
:1027580002F5806290420FD002F5806290420BD061
:10276800A2F59832904207D002F58062904203D0D9
:1027780002F58062904203D1CA6823F44073134380
:102788004A6923F08003134303608B68C3620B68B4
:102798008362064B984203D003F58063984201D1C7
:1027A8000B69036301234361704700BF00000140C8
:1027B8000040014010B50446A0B190F83D3003F048
:1027C800FF021BB980F83C2006F0ECF902232068D0
:1027D80084F83D30211DFFF787FF0123002084F88E
:1027E8003D3010BD012010BD90F83C3030B5012BB4
:1027F8004FF0020314D0046880F83D306268A36883
:102808000D68496822F0700223F080030B432A43C5
:102818006260A360012380F83D30002380F83C30DB
:10282800184630BD704770470368DA6822F4907222
:10283800DA605A6922F001025A61202380F83A309E
:102848007047000038B504460368C1681A692569ED
:1028580022F440520A431A61A268D9682A4365697A
:10286800C0692A4321F4164121F00C0102430A43AE
:10287800DA605A69A16922F440720A43B0F5004F40
:102888005A61224A24D1934203D002F580629342CE
:102898001BD1FFF75BFE19235843636821685B006F
:1028A8006424B0FBF3F0B0FBF4F504FB1503DB0084
:1028B8003233B3FBF4F303F007025B0002EB0512BB
:1028C80003F4F87313448B6038BDFFF727FEE2E783
:1028D800934202D00E4A934214D1FFF737FE1923D0
:1028E8005843636864229B00B0FBF3F02168B0FB97
:1028F800F2F402FB14031B013233B3FBF2F303EBD4
:102908000413E0E7FFF70AFEE9E700BF0010014003
:1029180000140140F8B504460E4617461D462168C6
:102928000B6836EA030301D10020F8BD6B1CF7D011
:1029380095B923680320DA6822F4D072DA605A69FC
:1029480022F001025A61202384F8393084F83A30A1
:10295800002384F83830F8BDFEF740FCC01B8542E0
:10296800DDD2E6E710B5044640B390F8393003F0FD
:10297800FF021BB980F8382006F02CF924232268BE
:1029880084F83930D368204623F40053D360FFF726
:1029980059FF236800201A6922F490421A615A6983
:1029A80022F02A025A61DA6842F40052DA602023DF
:1029B800E06384F8393084F83A3010BD012010BD46
:1029C8002DE9F0411F4690F839300446202B0D467A
:1029D80090464ED1002949D0002A47D090F8383087
:1029E800012B46D0012380F838300023C36321230C
:1029F80080F83930FEF7F2FB0646A4F82480A4F8E4
:102A08002680E38C9BB26BB93B4632464021204678
:102A1800FFF780FFA8B9202384F8380084F83930FC
:102A2800BDE8F081E38C3246013B9BB2E384A368A6
:102A38008021B3F5805F20463B460ED1FFF76AFF41
:102A480010B10320BDE8F0812B882268C3F3080386
:102A58005360236943B90235D3E7FFF75BFF0028CA
:102A6800EFD123682A785A600135CAE70120BDE80A
:102A7800F0810220BDE8F08138B50446134694F889
:102A88003920202A2AD139B333B394F83820012ABF
:102A980024D00122002584F838202122E384206BE9
:102AA800E56384F839200E4AA3842162C2630D4A83
:102AB800056502640C4AC26422680432FEF7A6FC6B
:102AC8006FF04002236828461A605A6984F8385023
:102AD80042F080025A6138BD012038BD022038BD5D
:102AE800872B0008B52B0008812C0008134690F8A6
:102AF8003A2073B5202A054638D1002934D0002B56
:102B080032D090F83820012A30D00122002480F8F1
:102B180038202222C4638162838580F83A20406B82
:102B2800134A2E68C263134A04650264124AC264D7
:102B38000A46311DFEF76AFC20462B6801941A6884
:102B480001925A6885F838400192019ADA6842F48D
:102B58008072DA605A6942F001025A615A6942F099
:102B680040025A6102B070BD0120FBE70220F9E77C
:102B7800BF2B0008752C0008812C0008704708B589
:102B88000368826B1B6813F480730AD1D3841368BB
:102B98005A6922F080025A61DA6842F04002DA602B
:102BA80008BD1046FFF7EAFF08BD704708B5806BFF
:102BB800FFF7FBFF08BD08B50368826B1B6813F4B9
:102BC800807310D1D3851368D96821F48071D960D6
:102BD800596921F001015961596921F04001596190
:102BE800202382F83A30104605F0D2FB08BD90F851
:102BF8003A3010B5222B36D183680169B3F5805F6E
:102C08000268836A23D15268E9B9C2F3080223F83B
:102C1800022B8362C48D013CA4B2C4858CB90368BD
:102C2800DA6822F02002DA60DA6822F48072DA6068
:102C38005A6922F001025A61202380F83A3005F0DF
:102C4800A7FB002010BDD2B223F8012BE1E721B980
:102C5800591C526881621A70DCE75268591C8162FB
:102C680002F07F02F7E7022010BD704708B5806BBD
:102C7800FFF7FBFF08BD7047816B08B50B685A6901
:102C880091F8390021280AD1120608D50022CA84F1
:102C9800DA6822F0C002DA60202281F839205B6904
:102CA80091F83A20222A06D15B0604D5002308466B
:102CB800CB85FFF7B9FDCB6B084643F01003CB6318
:102CC800FFF7D9FF08BD0000036870B51A6804460D
:102CD8001607D9685D6907D196065AD58D0658D565
:102CE800BDE87040FFF783BF15F0010502D111F46C
:102CF800907F4ED0D30705D5CE0542BFE36B43F096
:102D08000103E363500704D51DB1E36B43F00203ED
:102D1800E363930704D51DB1E36B43F00403E36356
:102D2800160704D51DB1E36B43F00803E363E36BB7
:102D3800002B66D0950604D5880602D52046FFF7F5
:102D480056FF236820465D69E26B110702D415F02F
:102D580040051AD0FFF768FD23685A69520610D556
:102D68005A69606B22F040025A6150B1254B0365E5
:102D7800FEF787FB002844D0606BBDE87040036D08
:102D880018472046FFF777FF70BDFFF774FFE5632C
:102D980070BD160627D50D0625D594F83920212AA9
:102DA8002FD1A268B2F5805F226A17D11188C1F3CA
:102DB80008015960216979B902322262E28C013A2C
:102DC80092B2E284EAB9DA6822F08002DA60DA685C
:102DD80042F04002DA6070BD0132EEE7511C216218
:102DE80012785A60EAE750060BD54A0609D5DA6820
:102DF800204622F04002DA60202384F83930FFF7B9
:102E0800BDFE70BD112E000808B50023806BC38578
:102E1800C384FFF730FF08BD014B1870704700BF2F
:102E280030020020014B1878704700BF30020020A4
:102E380010B50446087801F05FFA206010BD38B577
:102E4800044608780D4601F011FA2060687801F010
:102E58000DFA01462068FDF751FE2060A87801F0C0
:102E680005FA01462068FDF749FE2060E87801F080
:102E7800FDF901462068FDF741FE206038BD38B5F0
:102E8800044608780D4601F0C7FA2060687801F01A
:102E9800C3FA01462068FDF731FE2060A87801F0EA
:102EA80073FA01462068FDF729FE206038BD00004E
:102EB8000138122838D8DFE800F00A3737372237C8
:102EC800370E1215191C1F25282B2E3134001749CF
:102ED8001748FFF7ADBF17491748FFF7B0BF1749A5
:102EE8001748FAE717491848FFF7C9BF174918489C
:102EF800FAE718491848F7E718491948F4E719494B
:102F08001948E6E719491A48E7E71A491A48E4E769
:102F18001A491B48E8E71B491B48E5E71B491C48B9
:102F2800E2E71C491C48DFE7704700BFD60A0020CB
:102F3800F8010020D70A00200C020020DB0A00203C
:102F480010020020DF0A0020FC010020E20A002015
:102F580000020020E50A002004020020E80A002000
:102F680008020020EB0A002014020020EC0A0020CE
:102F780028020020F00A00202C020020F40A002079
:102F880018020020F70A00201C020020FA0A00207C
:102F980020020020FD0A0020240200200023DAB2CB
:102FA800815C01330029FAD1104670472DE9F047BA
:102FB8004FF0100A4FF020099EB001AF80460D4631
:102FC800144600215246384605AE05F068FF4A46C9
:102FD8000021304605F063FF4FF48053ADF83430DC
:102FE8004FF40063ADF836304FF40053ADF8383085
:102FF8004FF48043ADF83C304FF40043ADF83E3019
:103008000423ADF840300823ADF842304023ADF832
:1030180048308023ADF846A0ADF84490ADF84A306A
:10302800B8F1000F02D0404600F01BFA00224FF41E
:1030380078413B48FEF7DAFB0022FC213948FEF7CD
:10304800D5FB002D67D12A464FF400613448FEF7BE
:10305800CDFB0FAB93E8030016AB87E8030093E8BA
:103068000300012286E803004FF400512C48FEF7C4
:10307800BDFB14F0010218BF01224FF4804128481B
:10308800FEF7B4FB14F0020218BF01224FF400410E
:103098002348FEF7ABFB14F0040218BF01220421F9
:1030A8002048FEF7A3FB14F0080218BF01220821EC
:1030B8001C48FEF79BFB14F0100218BF01222021C8
:1030C8001848FEF793FB14F0200218BF01221021C4
:1030D8001448FEF78BFB14F0400218BF0122402170
:1030E8001048FEF783FB23064CBF012200228021F3
:1030F8000C48FEF77BFB00224FF400510848FEF70E
:1031080075FB55B901224FF4006105481EB0BDE8B2
:10311800F047FEF76BBB012296E70022F3E700BFFA
:10312800000C024000180240002138B5AF4C0C22B8
:103138000846FFF73BFFA07901F0DEF8AC4BAD4D38
:103148001860E07901F092F801462868FDF7D6FC8E
:103158002860207A01F08AF801462868FDF7CEFC3D
:103168002860607A01F082F801462868FDF7C6FCFD
:103178002860A07A01F07AF801462868FDF7BEFCBD
:103188002860E07A01F072F89B4D01462868FDF747
:10319800B5FC2860207B01F069F801462868FDF736
:1031A800ADFC2860607B01F061F801462868FDF7F6
:1031B800A5FC2860A07B01F059F801462868FDF7B6
:1031C8009DFC2860E07B01F027F98C4D01462868BA
:1031D800FDF794FC2860207C01F01EF90146286860
:1031E800FDF78CFC2860607C01F0CEF80146286869
:1031F800FDF784FC2860A07C01F00EF9804D0146A3
:103208002868FDF77BFC2860E07C01F005F90146A1
:103218002868FDF773FC2860207D01F0B5F80146A9
:103228002868FDF76BFC2860607D01F0F5F8754DA6
:1032380001462868FDF762FC2860A07D01F0ECF8E3
:1032480001462868FDF75AFC2860E07D01F09CF8EB
:1032580001462868FDF752FC2860207E01F0DCF862
:10326800694D01462868FDF749FC2860607E01F039
:10327800D3F801462868FDF741FC2860A07E01F0DC
:1032880083F801462868FDF739FC2860E07E01F0E4
:1032980033F85E4B5E4D1860207F00F0E7FF014673
:1032A8002868FDF72BFC2860607F00F0DFFF0146EF
:1032B8002868FDF723FC2860A07F00F0D7FF0146AF
:1032C8002868FDF71BFC2860E07F00F0CFFF01466F
:1032D8002868FDF713FC286094F8200000F0C6FF6A
:1032E8004C4D01462868FDF709FC286094F8210038
:1032F80000F0BCFF01462868FDF700FC286094F840
:10330800220000F0B3FF01462868FDF7F7FB2860AC
:1033180094F8230000F0AAFF01462868FDF7EEFBA9
:10332800286094F8240001F077F83B4D014628689E
:10333800FDF7E4FB286094F8250001F06DF80146DC
:103348002868FDF7DBFB286094F8260001F01CF8DC
:1033580001462868FDF7D2FB286094F8270001F0A1
:103368005BF82E4D01462868FDF7C8FB286094F8E5
:10337800280001F051F801462868FDF7BFFB2860D6
:1033880094F8290001F000F801462868FDF7B6FB1B
:10339800286094F82A0001F03FF8214D014628687A
:1033A800FDF7ACFB286094F82B0001F035F80146D6
:1033B8002868FDF7A3FB286094F82C0000F0E4FFD0
:1033C80001462868FDF79AFB286094F82D0001F063
:1033D80023F8144D01462868FDF790FB286094F8FF
:1033E8002E0001F019F801461EE000BFD00A0020A7
:1033F800F80100200C02002010020020FC0100202F
:10340800000200200402002008020020140200200C
:10341800280200202C020020180200201C02002094
:1034280020020020240200202868FDF767FB28609E
:1034380094F82F0000F0A8FF01462868FDF75EFB0E
:10344800286038BD00210F220846FFF7AFBD0021D4
:103458000C220846FFF7AABD002101220846FFF703
:10346800A5BD002101280CBF8022C0220846FFF715
:103478009DBD00002DE9F04F10252024A1B00DF1CD
:103488000C0A904607462A468946504600210DF107
:103498001C0B05F004FD22460021584605F0FFFCF0
:1034A8004FF48053ADF83C304FF40063ADF83E3034
:1034B8004FF40053ADF840304FF48043ADF844303A
:1034C8004FF40043ADF846300423ADF848300823E4
:1034D800ADF84A304023ADF8503080234046ADF86F
:1034E8004E50ADF84C40ADF85230FFF757FD464608
:1034F800504D514C0190A6EB0803019ADBB29A4259
:1035080002D821B0BDE8F08F002F40F08780002757
:1035180000224FF478412846FEF768F90022FC2182
:103528002046FEF763F9B9F1000F7ED14A464FF401
:1035380000612846FEF75AF911AB93E8030018AB6F
:103548008AE8030093E8030001228BE803004FF4A4
:1035580000512846FEF74AF916F8012B4FF480412E
:1035680012F0010218BF01222846FEF73FF916F8AB
:10357800012C4FF4004112F0020218BF0122284624
:10358800FEF734F916F8012C042112F0040218BFD2
:1035980001222046FEF72AF916F8012C082112F01C
:1035A800080218BF01222046FEF720F916F8012C60
:1035B800202112F0100218BF01222046FEF716F94A
:1035C80016F8012C102112F0200218BF0122204603
:1035D800FEF70CF916F8012C402112F0400218BF32
:1035E80001222046FEF702F916F9013C8021002B42
:1035F800B4BF012200222046FEF7F8F800224FF45B
:1036080000512846FEF7F2F8B9F1000F0FD1012258
:103618004FF400612846FEF7E9F86CE73846FFF7F3
:1036280020FF022F3FF473AF72E701227FE70022E9
:10363800EEE700BF000C024000180240014B18786A
:10364800704700BF3202002008B5FFF700FFFFF700
:1036580003FF0C4A01210020FFF70CFF1022012173
:103668000020FFF7A3FC084A0849104606F0D6F9DF
:10367800012102460220FFF7FDFE0022044B1A70CA
:1036880008BD00BFC9BB000834020020D9BB000830
:103698003202002010B5FFF7DAFEFFF7DDFE0F4A11
:1036A80001210020FFF7E6FE102201210020FFF78C
:1036B8007DFC0B4B0B4C1868FCF7EEFE0B460246E4
:1036C8000949204606F086F9224601210220FFF723
:1036D800D1FE0122054B1A7010BD00BF9EBB000829
:1036E800F801002044020020ADBB0008320200208F
:1036F80010B5FFF7ACFEFFF7AFFE11220121002045
:10370800FFF754FC0E4A01210020FFF7B3FE1022F8
:1037180001210020FFF74AFC0A4B0B4C1868FCF704
:10372800BBFE0B4602460949204606F053F92246DD
:1037380001210220FFF79EFE0222054B1A7010BDE0
:10374800E5BB00080C02002054020020ADBB0008B5
:103758003202002010B5FFF77AFEFFF77DFE112236
:1037680001210020FFF722FC0C4A01210020FFF76D
:1037780081FE0B4B0B4C1868FCF78EFE0B4602467D
:103788000949204606F026F9224601210220FFF7C2
:1037980071FE0322054B1A7010BD00BFBDBB0008A7
:1037A800FC01002064020020ADBB000832020020AA
:1037B80008B5FFF74CFEFFF74FFE1122012100204C
:1037C800FFF7F4FB094A01210020FFF753FE084ADE
:1037D8000849104606F022F9012102460220FFF7A7
:1037E80049FE0422044B1A7008BD00BF0FBC000834
:1037F80074020020D9BB00083202002010B5FFF780
:1038080026FEFFF729FE0F4A01210020FFF732FEAE
:10381800102201210020FFF7C9FB0B4B0B4C186845
:10382800FCF73AFE0B4602460949204606F0D2F854
:10383800224601210220FFF71DFE0522054B1A70C2
:1038480010BD00BFF4BB0008140200208402002051
:10385800ADBB00083202002010B5FFF7F8FDFFF7F6
:10386800FBFD112201210020FFF7A0FB0E4A0121D8
:103878000020FFF7FFFD102201210020FFF796FB33
:103888000A4B0B4C1868FCF707FE0B460246094921
:10389800204606F09FF8224601210220FFF7EAFDA4
:1038A8000622054B1A7010BD1BBC00082802002018
:1038B80094020020ADBB00083202002010B5FFF7CB
:1038C800C6FDFFF7C9FD112201210020FFF76EFB9D
:1038D8000C4A01210020FFF7CDFD0B4B0B4C18685B
:1038E800FCF7DAFD0B4602460949204606F072F855
:1038F800224601210220FFF7BDFD0722054B1A7061
:1039080010BD00BF03BC000818020020A40200205C
:10391800ADBB000832020020F8B515460C46074634
:10392800FFF790FD21682846FDF7E8F8104E206063
:1039380031460546FDF756FA08B12660F8BD00265F
:1039480028463146FDF730FA0028F6D12846FCF71C
:10395800A3FD0B4602460749074806F03BF8064A0E
:1039680001210220FFF786FD044B1F70F8BD00BF40
:103978000000F041ADBB0008B40200203202002074
:10398800F8B515460C460746FFF75CFD2168284642
:10399800FDF7B4F8104E206031460546FDF722FACF
:1039A80008B12660F8BD002628463146FDF7FCF927
:1039B8000028F6D12846FCF76FFD0B46024607495A
:1039C800074806F007F8064A01210220FFF752FDD2
:1039D800044B1F70F8BD00BF0000F042ADBB0008EB
:1039E800C402002032020020F8B515460C460746EE
:1039F800FFF728FD21682846FDF780F8104E206063
:103A080031460546FDF7EEF908B12660F8BD0026F7
:103A180028463146FDF7C8F90028F6D12846FCF7B4
:103A28003BFD0B4602460749074805F0D3FF064A07
:103A380001210220FFF71EFD044B1F70F8BD00BFD7
:103A48000000B442ADBB0008D402002032020020BE
:103A580038B504460D46FFF7FAFCFFF7FDFC082CC5
:103A680001D00E2C1AD1154A01210020FFF702FDC2
:103A7800102201210020FFF799FA2868FCF70CFDB5
:103A88000B4602460E490F4805F0A4FF0D4A0121D6
:103A98000220FFF7EFFC0C4B1C7038BD092C01D03D
:103AA8000F2CEAD1112201210020FFF77FFA074AE3
:103AB80001210020FFF7DEFCDFE700BF7EBB000826
:103AC800ADBB0008E4020020320200208EBB0008D3
:103AD80038B504460D46FFF7BAFCFFF7BDFC0A2CC3
:103AE80001D0102C1AD1204A01210020FFF7C2FC76
:103AF800102201210020FFF759FA2868FCF7CCFCB6
:103B08000B46024619491A4805F064FF184A012174
:103B18000220FFF7AFFC174B1C7038BD0B2C01D0EF
:103B2800112C06D1112201210020FFF73FFA124A79
:103B3800DAE70C2C01D0122C06D111220121002029
:103B4800FFF734FA0D4ACFE70D2C01D0132CD4D14E
:103B5800112201210020FFF729FA094A012100203A
:103B6800FFF788FCC9E700BF41BB0008ADBB0008F0
:103B7800F40200203202002051BB000860BB00089C
:103B88006FBB000838B5AD4D04462B789BB968B9B2
:103B9800FFF762FC2046AA4A0121FFF76BFCBDE84B
:103BA8003840A84A01210220FFF764BCFFF74CFD0A
:103BB80001232B7038BD022803D1BDE83840FFF738
:103BC80043BDA14B1D782846FFF772F9212D00F25D
:103BD8007081DFE815F022003800450058002F00FA
:103BE800620071007E00850093009E00AC00B90061
:103BF800C600CE00DD00E500F000FD000A0112015C
:103C08002D016F018701B301DD010802330248026B
:103C180061027A02A502EA021503042C03D1BDE869
:103C28003840FFF7C5BD052C40F04381BDE838405A
:103C3800FFF730BD032CC0D0052C40F03A81BDE819
:103C48003840FFF7DBBD042C03D1BDE83840FFF74F
:103C58004FBD052C40F02D8100227C49142027E01F
:103C6800042C03D1BDE83840FFF774BD032CDDD028
:103C7800052C05D108207649BDE83840FFF7E8BE95
:103C8800012C9AD038BD032CDFD0052CF8D10A209E
:103C98007049BDE83840FFF71BBF042C03D1BDE8CD
:103CA8003840FFF7D9BD052CEAD100221B206A490C
:103CB800BDE83840FFF730BE042C03D1BDE83840DA
:103CC800FFF7FCBD032CBAD0052CD9D163490E20CF
:103CD800D2E7032CE3D0052CD2D161491020D8E7D4
:103CE800042C02D15F490920C6E7052C03D1002224
:103CF8005749152009E0012C98D038BD032CB9D0BC
:103D0800052CF8D1002216205649BDE83840FFF7A7
:103D180037BE042C02D154490B20BAE7052CEAD14E
:103D280000224C491720BDE83840FFF75DBE042C3F
:103D380002D14E490C20ACE7032CA8D0052CDAD1CF
:103D4800002249491820EEE7042C02D148490D20E9
:103D58009FE7032CDFD0052CCDD100224349192041
:103D6800E1E7032CE5D0052CC5D1002240491A20F3
:103D7800D9E7042C02D13F490F207DE7052C03D158
:103D8800002236491C20C0E7012C3FF458AF38BD4B
:103D9800032C9BD0052CF7D1002236491D20B4E70F
:103DA800042C02D13449112073E7052CECD10022F0
:103DB8002B491E20B7E7042C02D13049122068E7AE
:103DC800032C8AD0052CDFD100222B491F20AAE71B
:103DD800042C02D12A4913205BE7032CE2D0052CDE
:103DE800D2D10022254920209DE7032CE5D0052CBF
:103DF800CAD100222249212095E7032C02D14FF095
:103E08007C522AE7042C02D14FF03F4225E7052CCB
:103E18007FF471AF0D4C002221461420FFF77CFD82
:103E28000121206800F0B6FC0122164B1A7038BD3B
:103E3800032C29D14FF07C525AE700BF33020020EF
:103E480020BB000830BB000832020020F801002027
:103E58000C020020FC01002014020020280200208F
:103E68001802002010020020000200200402002096
:103E7800080200202C0200201C0200202002002042
:103E88002402002031020020042C02D14FF03F42CE
:103E98002EE7052C0AD1A84C0221206800F0AAFCC4
:103EA800002221461520FFF76BFDBDE7012C3FF4EA
:103EB800E1AE38BD032C02D14FF07C5223E7042C2D
:103EC80002D14FF03F421EE7052C08D19B4C03213D
:103ED800206800F08FFC002221461620E3E7012C21
:103EE800E7D1FFE6032C0CD1954C96492068FCF7E6
:103EF80065FF18B14FF07E52214613E74FF07C5210
:103F0800FAE7042C0AD18E4C8E492068FCF756FF3C
:103F180008B18D4AF0E74FF03F42EDE7052C0AD192
:103F2800874C0421206800F0D9FC00222146172084
:103F3800FFF75AFD78E7012CBBD1A8E6032C0CD17A
:103F4800824C80492068FCF739FF18B14FF07E5247
:103F58002146F7E64FF07C52FAE7042C0AD17B4C55
:103F680078492068FCF72AFF08B1774AF0E74FF054
:103F78003F42EDE7052C08D1744D2146286800F032
:103F8800ADFC002229461820D2E7012C91D1C2E6C7
:103F9800032C0CD16E4C6B492068FCF70FFF18B14D
:103FA8004FF07E522146DAE64FF07C52FAE7042CB5
:103FB8000AD1674C63492068FCF700FF08B1624AE0
:103FC800F0E74FF03F42EDE7052C08D1604C0621A1
:103FD800206800F083FC002221461920A8E7012C64
:103FE8007FF467AFA5E6032C0CD15A4C55492068DD
:103FF800FCF7E4FE18B14FF07E522146B7E64FF0C9
:104008007C52FAE7042C0AD1524C4E492068FCF73E
:10401800D5FE08B14C4AF0E74FF03F42EDE7052CDA
:1040280008D14C4C0721206800F058FC002221469A
:104038001A207DE7012C7FF43CAF87E6032C02D1E0
:104048004FF07C5232E6042C02D14FF03F422DE66D
:10405800052C7FF499AE404C002221461B20FFF727
:104068005BFC0821DDE6032C02D14FF07C5288E688
:10407800042C02D14FF03F4283E6052C08D1374C7F
:104088000921206800F0B6FB002221461C200AE71F
:10409800012C7FF40EAF19E6032C02D14FF07C52AD
:1040A8007BE6042C02D14FF03F4276E6052C08D17E
:1040B8002B4C0A21206800F09DFB002221461D2080
:1040C800F1E6012C7FF4F5AE55E6032C0CD1254C16
:1040D8001C492068FCF772FE18B14FF07E52214649
:1040E80067E64FF07C52FAE7042C0AD11D4C1549BB
:1040F8002068FCF763FE08B1134AF0E74FF03F422F
:10410800EDE7052C08D1174C0B21206800F0E6FBE1
:10411800002221461E200BE7012C7FF4CAAEDCE505
:10412800032C26D1104C07492068FCF747FEE8B15C
:104138004FF07E52214649E60C0200201002002072
:10414800FC01002000007042000080BF0002002037
:104158000402002008020020140200202802002087
:104168002C020020180200201C0200204FF07C5274
:10417800E0E7042C0AD1384C38492068FCF71EFEC9
:1041880008B1374AD6E74FF03F42D3E7052C08D1AC
:10419800314C0C21206800F0A1FB002221461F2091
:1041A800C6E6012C7FF485AEFCE5032C0CD12D4C22
:1041B8002A492068FCF702FE18B14FF07E522146CA
:1041C80011E64FF07C52FAE7042C0AD1254C23491A
:1041D8002068FCF7F3FD08B1214AF0E74FF03F42B1
:1041E800EDE7052C08D11F4C0D21206800F076FB67
:1041F8000022214620209BE6012C7FF45AAEDCE504
:10420800032C0CD1184C15492068FCF7D7FD18B1C0
:104218004FF07E522146EEE54FF07C52FAE7042C2F
:104228000AD1114C0D492068FCF7C8FD08B10C4AA9
:10423800F0E74FF03F42EDE7052C08D10A4C0E217C
:10424800206800F04BFB00222146212070E6012C5B
:104258007FF42FAEBEE500BF1C02002000007042B4
:10426800000080BF20020020240200202DE9F84F22
:10427800A8B100F07E044FF0834600204FF082473B
:104288004FF081484FF080494FF07E5A4FF07C5BE9
:10429800184D34B90021FCF731FCBDE8F88F002037
:1042A800F8E7A10705D5594604F0FD04FCF726FCFC
:1042B800EFE7620703D504F0FB045146F6E723074E
:1042C80003D504F0F7044946F0E7E10603D504F006
:1042D800EF044146EAE7A20603D504F0DF043946B5
:1042E800E4E7630647BF04F0BF04314604F0FD0469
:1042F8002946DBE70000FC412DE9F047A8B1C0439F
:104308004FF0834500F03F044FF0824600204FF005
:1043180081474FF080484FF07E594FF07C5A34B9AE
:104328000021FCF7EBFBBDE8F0870020F8E7E10788
:1043380005D5514604F0FE04FCF7E0FBEFE7A207C1
:1043480003D504F0FD044946F6E7630703D504F0F6
:10435800FB044146F0E7210703D504F0F70439468A
:10436800EAE7E20603D504F0EF043146E4E7A306E2
:1043780003D504F0DF042946DEE70249FCF7BEFB5B
:10438800CEE700BF0000FC412DE9F84F00F03F04E4
:104398004FF07C5500204FF07E564FF080474FF08D
:1043A80081484FF082494FF0834ADFF868B03F2CCC
:1043B80003D15946FCF7A2FB0024A10605D55146B6
:1043C80004F01F04FCF79AFBF1E7E20603D504F0BA
:1043D8002F044946F6E7230703D504F0370441467E
:1043E800F0E7610703D504F03B043946EAE7A20782
:1043F80003D504F03D043146E4E7E30703D504F0B0
:104408003E042946DEE7002CD1D10021FCF776FBDB
:10441800BDE8F88F0000FC41C0432DE9F84300F0E7
:104428001F044FF0834500204FF082464FF081472C
:104438004FF080484FF07E5924B90021FCF75EFB0D
:10444800BDE8F883E20705D5494604F01E04FCF7E9
:1044580055FBF1E7A30703D504F01D044146F6E731
:10446800610703D504F01B043946F0E7220703D59A
:1044780004F017043146EAE7E30603D504F00F0415
:104488002946E4E714F01E0F14BF02490249FCF75D
:1044980035FBD2E70000F8410000FC412DE9F84F58
:1044A8008346002400254FF083464FF082474FF0A3
:1044B80081484FF080494FF07E5A29465846FCF70C
:1044C80069FC002852D12B495846FCF763FC60B9B7
:1044D80031465846FCF77CFC50B158463146FCF74B
:1044E8000BFB44F040048346E7E77E24AB46E4E751
:1044F80039465846FCF76CFC38B158463946FCF743
:10450800FBFA44F020048346D7E741465846FCF7B7
:104518005FFC38B158464146FCF7EEFA44F0100407
:104528008346CAE749465846FCF752FC38B1584614
:104538004946FCF7E1FA44F008048346BDE75146D2
:104548005846FCF745FC38B158465146FCF7D4FAB2
:1045580044F004048346B0E74FF07C515846FCF71A
:1045680037FC0028A9D044F00204BFE72046BDE884
:10457800F88F00BF0000FC412DE9F74F83463F2428
:1045880000254FF083464FF082474FF081484FF0A7
:1045980080494FF07E5A29465846FCF7FBFB0190AC
:1045A800002853D12B495846FCF7F4FB019A60B90F
:1045B80031465846FCF70CFC50B158463146FCF7DA
:1045C8009BFA04F01F048346E5E71446AB46E2E78E
:1045D80039465846FCF7FCFB38B158463946FCF7D3
:1045E8008BFA04F02F048346D5E741465846FCF77A
:1045F800EFFB38B158464146FCF77EFA04F0370421
:104608008346C8E749465846FCF7E2FB38B15846A6
:104618004946FCF771FA04F03B048346BBE7514670
:104628005846FCF7D5FB38B158465146FCF764FAB2
:1046380004F03D048346AEE74FF07C515846FCF742
:10464800C7FB0028A7D004F03E04BFE7204603B00C
:10465800BDE8F08F0000FC412DE9F84F0546002425
:1046680000264FF083474FF082484FF081494FF0C2
:10467800804A4FF07E5B31462846FCF78BFB0028CA
:1046880058D12E492846FCF785FB60B9394628469B
:10469800FCF79EFB50B128463946FCF72DFA44F04A
:1046A80020040546E7E73F243546E4E74146284627
:1046B800FCF78EFB38B128464146FCF71DFA44F05A
:1046C80010040546D7E749462846FCF781FB38B170
:1046D80028464946FCF710FA44F008040546CAE79C
:1046E80051462846FCF774FB38B128465146FCF77A
:1046F80003FA44F004040546BDE759462846FCF78A
:1047080067FB38B128465946FCF7F6F944F002042D
:104718000546B0E74FF07C512846FCF759FB0028C6
:10472800A9D028464FF07C51FCF7E6F944F0010483
:104738000546A0E72046BDE8F88F00BF0000FC4111
:1047480003461F202BB31F2B06D00F2B06D9103B77
:10475800DBB200F00F00F5E700207047072B04D903
:10476800083BDBB200F01700ECE7032B04D9043B4D
:10477800DBB200F01B00E5E7012B89BF023B03F128
:10478800FF33DBB200F01D009CBFDBB200F01E005F
:10479800D8E770471FB5002302938DF80C30BE236D
:1047A8008DF8043004238DF805108DF80630FFF7D6
:1047B800E3FE3F238DF8070006210DF105008DF873
:1047C80008308DF809308DF80A30EB2404F03DF9F3
:1047D800074A8DF80B008DF80C4001AB03CB14721F
:1047E800106051600120FEF717FB04B010BD00BF38
:1047F800D90300201FB50023019302938DF80C30D4
:10480800BE238DF8043004238DF805102F49044683
:104818008DF80630FCF7E6FA18B378232B492046C2
:104828008DF807308DF808308DF80930FCF764F9F9
:10483800FFF734FE8DF80A0006210DF1050004F09B
:1048480004F9EB24224A8DF80B008DF80C4001ABDB
:1048580003CB1472106051600120FEF7DDFA04B03A
:1048680010BD1C492046FCF7BDFA88B119492046FD
:10487800FCF742F90446FFF711FE782320468DF82D
:1048880007308DF80830FFF709FE8DF80900D3E7E7
:1048980011492046FCF7A6FA58B178230E4920465C
:1048A8008DF80730FCF728F9FFF7F8FD8DF80800B8
:1048B800C2E700212046FCF78BFA0028BCD020462E
:1048C800FFF7ECFD8DF80700B6E700BF0000B44223
:1048D800D9030020000070420000F0411FB50023FA
:1048E800019302938DF80C30BE238DF80430032316
:1048F8008DF80510264904468DF80630FCF772FA43
:1049080000B30123224920468DF807308DF808307E
:10491800FCF7F2F8FFF7A0FE8DF8090005210DEB72
:10492800010004F092F8EB231A4A8DF80B308DF849
:104938000A0001AB03CB106051600120FEF76CFA4E
:1049480004B010BD14492046FCF742FA70B10123A7
:10495800114920468DF80730FCF7CEF8FCF74CFAE1
:10496800C0B2FFF7EDFE8DF80800D7E7002120461A
:10497800FCF72EFA0028D1D02046FCF73DFAC0B249
:10498800FFF7DEFE1F238DF807008DF80830C5E716
:1049980000007042D90300200000F041F8B5064637
:1049A800002954D0012955D0022956D0032957D0BF
:1049B800042914BF4FF480654FF48045002229462E
:1049C8002948FCF713FF0120FCF70EFC0824264FAA
:1049D80016F0010218BF01224FF400713846FCF7A7
:1049E80005FF01224FF480711F48FCF7FFFE0120EC
:1049F800FCF7FAFB00224FF480711B48FCF7F6FE27
:104A0800013C0120FCF7F0FB14F0FF044FEA5606C6
:104A1800DED122464FF480711348FCF7E7FE2246A8
:104A28004FF400711048FCF7E1FE0120FCF7DCFBB5
:104A3800294601220C48FCF7D9FE0120FCF7D4FBDB
:104A480022462946BDE8F8400748FCF7CFBE4FF498
:104A58008065B3E74FF40065B0E74FF48055ADE7E4
:104A68004FF40055AAE700BF001002402DE9F041BD
:104A780005460F4600295BD001295DD002295ED08A
:104A880003295FD0042931481ABF4FF480660020FB
:104A98004FF4007600223146FCF7A8FE0120FCF70F
:104AA800A3FB0824DFF8A88015F0010218BF012233
:104AB8004FF400514046FCF799FE01224FF4805113
:104AC8002348FCF793FE0120FCF78EFB00224FF4ED
:104AD80080511F48FCF78AFE013C0120FCF784FB4B
:104AE80014F0FF044FEA5505DED122464FF48051F9
:104AF8001748FCF77BFE22464FF400511448FCF798
:104B080075FE0120FCF770FB114D104B3146002F4C
:104B180018BF1D4601222846FCF768FE0120FCF755
:104B280063FB224631462846BDE8F041FCF75EBEED
:104B380007484FF48046ADE704484026AAE70348F3
:104B48008026A7E701482026A4E700BF000402400A
:104B580000180240F8B50646002949D001294AD074
:104B680002294BD003294CD0042914BF4FF4806587
:104B78004FF480450624244F16F0200218BF012266
:104B88004FF400713846FCF731FE01224FF4807172
:104B98001D48FCF72BFE0120FCF726FB00224FF4F2
:104BA80080711948FCF722FE013C01207600FCF7D1
:104BB8001BFB14F0FF04F6B2DED122464FF48071DD
:104BC8001148FCF713FE22464FF400710E48FCF71B
:104BD8000DFE294601220C48FCF708FE0120FCF7CF
:104BE80003FB22462946BDE8F8400748FCF7FEBD0E
:104BF8004FF48065BEE74FF40065BBE74FF480557E
:104C0800B8E74FF40055B5E7001002402DE9F04130
:104C18000546884600294ED001294FD002294FD099
:104C280003294FD004290CBF4FF40077002706242E
:104C3800254E15F0200218BF01224FF400513046CE
:104C4800FCF7D4FD01224FF480513046FCF7CEFD2D
:104C58000120FCF7C9FA00224FF480513046FCF7D6
:104C6800C5FD013C01206D00FCF7BEFA14F0FF04FD
:104C7800EDB2DED122464FF480511348FCF7B6FD61
:104C8800114D124B2246B8F1000F18BF1D464FF4C4
:104C980000512846FCF7AAFD394601222846FCF7B0
:104CA800A5FD0120FCF7A0FA224639462846BDE8B2
:104CB800F041FCF79BBD4FF48047B8E74027B6E7C3
:104CC8008027B4E72027B2E700180240000402401A
:104CD80070B500224FF4004105462748FCF786FDD1
:104CE80000224FF480412448FCF780FD00224FF455
:104CF80000512148FCF77AFD08241F4E2B064CBFB3
:104D0800012200224FF480413046FCF76FFD01225A
:104D18004FF400511848FCF769FD0120FCF764FACC
:104D280000224FF400511448FCF760FD013C0120BB
:104D38006D00FCF759FA14F0FF04EDB2DED1012240
:104D48004FF400410C48FCF751FD0120FCF74CFAE8
:104D580022464FF400410848FCF748FD22464FF42C
:104D680080410548FCF742FD2246BDE870404FF4FB
:104D780000510148FCF73ABD0014024070B500220A
:104D88004FF4007105462448FCF730FD00228021CD
:104D98002248FCF72BFD002240212048FCF726FD85
:104DA80008241E4E2B064CBF0122002280213046CB
:104DB800FCF71CFD012240211848FCF717FD0120D3
:104DC800FCF712FA002240211448FCF70FFD013CC1
:104DD80001206D00FCF708FA14F0FF04EDB2E1D1F0
:104DE80001224FF400710C48FCF700FD0120FCF78C
:104DF800FBF922464FF400710748FCF7F7FC2246FE
:104E080080210648FCF7F2FC2246BDE870404021AC
:104E18000248FCF7EBBC00BF00180240000C02403F
:104E280038B504460D4610F0100218BF01221021B3
:104E38002248FCF7DBFC14F0080218BF012280218D
:104E48001F48FCF7D3FC14F0040218BF01224021CC
:104E58001B48FCF7CBFC14F0020218BF01222021EA
:104E68001748FCF7C3FC14F0010218BF01221021F7
:104E78001348FCF7BBFC8DB9012220210F48FCF731
:104E8800B5FC0120FCF7B0F92A4620210B48FCF7B5
:104E9800ADFCBDE838400120FCF7A6B9012D0BD1C7
:104EA8002A4629460748FCF7A1FC2846FCF79CF946
:104EB800002229460348EAE738BD00BF000802403F
:104EC800000002400004024038B504460D4610F0C8
:104ED800100218BF012202212348FCF787FC14F0B6
:104EE800080218BF012201211F48FCF77FFC14F0BB
:104EF800040218BF01224FF480511C48FCF776FCCD
:104F080014F0020218BF01224FF400611748FCF7A1
:104F18006DFC14F0010218BF01224FF480611348A0
:104F2800FCF764FC8DB9012204210F48FCF75EFCF4
:104F38000120FCF759F92A4604210B48FCF756FCD6
:104F4800BDE838400120FCF74FB9012D0AD12A46A7
:104F580008210548FCF74AFC2846FCF745F90022D9
:104F68000821EAE738BD00BF000C024000080240F3
:104F78002DE9F047164E044640213046FCF730FC38
:104F8800144D814602212846FCF72AFC8021074659
:104F98003046FCF725FC042182462846FCF720FC15
:104FA8004FF4807180463046FCF71AFC082106460B
:104FB8002846FCF715FC2670E07084F801A084F8F8
:104FC800029084F8048067712046BDE8F08700BF2E
:104FD800001402400008024007B502AB03E90300D1
:104FE8009DF8023013B19DF8053063BB00220421FF
:104FF8001F48FCF7FBFB012208211D48FCF7F6FBC4
:105008009DF8013013B19DF804301BBB002210211C
:105018001748FCF7EBFB012220211548FCF7E6FBBB
:105028009DF8003013B19DF80330D3B90022012157
:105038000F48FCF7DBFB012202210D4803B05DF8A5
:1050480004EBFCF7D3BB012204210948FCF7CEFB93
:105058000022D1E7012210210548FCF7C7FB0022F6
:10506800DAE7012202481146FCF7C0FB0022E3E719
:10507800001002400A4601460148FDF7FDBC00BF8A
:10508800C80F002084B070B504AC84E80F00BE22BD
:10509800124C149822704278E11C6270857804AA38
:1050A800A57014AE52F8043BB24241F8043BF9D162
:1050B800817801300231C9B203F0C7FCEB222544E4
:1050C800E870A378054823441A71A1780531C9B25C
:1050D800FFF7D0FFBDE8704004B0704768030020B8
:1050E80084B070B59AB01EAC84E80F006422002129
:1050F80001A89DF8B8502EAE03F0D1FE1EAA01AB50
:105108001C4610685168083203C4B2422346F7D1DE
:105118003F2D00F2E680DFE805F020272A2D303306
:1051280036393C3F4245484B4E5154575A5D6063AF
:1051380066696C6F7275787B7E8184878A8D90939F
:1051480096999C9FA2A5A8ABAEB1B4B7BABDC0C38F
:10515800C6C9CCCFD2D5D8DBDEE19DF878001AB02D
:10516800BDE8704004B070479DF87900F7E79DF8F6
:105178007A00F4E79DF87B00F1E79DF87C00EEE704
:105188009DF87D00EBE79DF87E00E8E79DF87F003D
:10519800E5E79DF88000E2E79DF88100DFE79DF8EC
:1051A8008200DCE79DF88300D9E79DF88400D6E704
:1051B8009DF88500D3E79DF88600D0E79DF8870025
:1051C800CDE79DF88800CAE79DF88900C7E79DF8F4
:1051D8008A00C4E79DF88B00C1E79DF88C00BEE704
:1051E8009DF88D00BBE79DF88E00B8E79DF88F000D
:1051F800B5E79DF89000B2E79DF89100AFE79DF8FC
:105208009200ACE79DF89300A9E79DF89400A6E703
:105218009DF89500A3E79DF89600A0E79DF89700F4
:105228009DE79DF898009AE79DF8990097E79DF803
:105238009A0094E79DF89B0091E79DF89C008EE703
:105248009DF89D008BE79DF89E0088E79DF89F00DC
:1052580085E79DF8A00082E79DF8A1007FE79DF80B
:10526800A2007CE79DF8A30079E79DF8A40076E703
:105278009DF8A50073E79DF8A60070E79DF8A700C4
:105288006DE79DF8A8006AE79DF8A90067E79DF813
:10529800AA0064E79DF8AB0061E79DF8AC005EE703
:1052A8009DF8AD005BE79DF8AE0058E79DF8AF00AC
:1052B80055E79DF8B00052E79DF8B1004FE79DF81B
:1052C800B2004CE79DF8B30049E79DF8B40046E703
:1052D8009DF8B50043E79DF8B60040E79DF8B70094
:1052E8003DE7024804F0B8FA002038E729BC000876
:1052F80084B070B59AB01EAC84E80F006422002117
:1053080001A89DF8B8502EAE03F0C9FD1EAA01AB46
:105318001C4610685168083203C4B2422346F7D1CC
:105328007E2D00F24581DFE815F0400143013D0183
:1053380043013A014301370143013401430131017B
:1053480043012E0143012B0143012801430125019B
:105358004301220143011F0143011C0143011901BB
:1053680043011601430113014301100143010D01DB
:1053780043010A01430107014301040143010101FB
:105388004301FE004301FB004301F8004301F5001F
:105398004301F2004301EF004301EC004301E9003F
:1053A8004301E6004301E3004301E0004301DD005F
:1053B8004301DA004301D7004301D4004301D1007F
:1053C8004301CE004301CB004301C8004301C5009F
:1053D8004301C2004301BF004301BC004301B900BF
:1053E8004301B6004301B3004301B0004301AD00DF
:1053F8004301AA004301A7004301A4004301A100FF
:1054080043019E0043019B0043019800430195001E
:105418004301920043018F0043018C00430189003E
:105428004301860043017F009DF878001AB0BDE86B
:10543800704004B070479DF87900F7E79DF87A004E
:10544800F4E79DF87B00F1E79DF87C00EEE79DF816
:105458007D00EBE79DF87E00E8E79DF87F00E5E733
:105468009DF88000E2E79DF88100DFE79DF8820063
:10547800DCE79DF88300D9E79DF88400D6E79DF81E
:105488008500D3E79DF88600D0E79DF88700CDE733
:105498009DF88800CAE79DF88900C7E79DF88A004B
:1054A800C4E79DF88B00C1E79DF88C00BEE79DF826
:1054B8008D00BBE79DF88E00B8E79DF88F00B5E733
:1054C8009DF89000B2E79DF89100AFE79DF8920033
:1054D800ACE79DF89300A9E79DF89400A6E79DF82E
:1054E8009500A3E79DF89600A0E79DF897009DE733
:1054F8009DF898009AE79DF8990097E79DF89A001B
:1055080094E79DF89B0091E79DF89C008EE79DF835
:105518009D008BE79DF89E0088E79DF89F0085E732
:105528009DF8A00082E79DF8A1007FE79DF8A20002
:105538007CE79DF8A30079E79DF8A40076E79DF83D
:10554800A50073E79DF8A60070E79DF8A7006DE732
:105558009DF8A8006AE79DF8A90067E79DF8AA00EA
:1055680064E79DF8AB0061E79DF8AC005EE79DF845
:10557800AD005BE79DF8AE0058E79DF8AF0055E732
:105588009DF8B00052E79DF8B1004FE79DF8B200D2
:105598004CE79DF8B30049E79DF8B40046E79DF84D
:1055A800B50043E79DF8B60040E79DF8B7003DE732
:1055B800024804F051F9002038E700BF29BC000870
:1055C80084B008B50DF1080E8EE80F009DF848303C
:1055D8003F2B00F2E580DFE803F0E0DDDAD7D4D135
:1055E800CECBC8C5C2BFBCB9B6B3B0ADAAA7A4A13B
:1055F8009E9B9895928F8C898683807D7A7774712B
:105608006E6B6865625F5C595653504D4A4744411A
:105618003E3B3835322F2C2926209DF80800BDE85E
:10562800084004B070479DF80900F8E79DF80A00A3
:10563800F5E79DF80B00F2E79DF80C00EFE79DF801
:105648000D00ECE79DF80E00E9E79DF80F00E6E78E
:105658009DF81000E3E79DF81100E0E79DF81200BF
:10566800DDE79DF81300DAE79DF81400D7E79DF809
:105678001500D4E79DF81600D1E79DF81700CEE78E
:105688009DF81800CBE79DF81900C8E79DF81A00A7
:10569800C5E79DF81B00C2E79DF81C00BFE79DF811
:1056A8001D00BCE79DF81E00B9E79DF81F00B6E78E
:1056B8009DF82000B3E79DF82100B0E79DF822008F
:1056C800ADE79DF82300AAE79DF82400A7E79DF819
:1056D8002500A4E79DF82600A1E79DF827009EE78E
:1056E8009DF828009BE79DF8290098E79DF82A0077
:1056F80095E79DF82B0092E79DF82C008FE79DF821
:105708002D008CE79DF82E0089E79DF82F0086E78D
:105718009DF8300083E79DF8310080E79DF832005E
:105728007DE79DF833007AE79DF8340077E79DF828
:10573800350074E79DF8360071E79DF837006EE78D
:105748009DF838006BE79DF8390068E79DF83A0046
:1057580065E79DF83B0062E79DF83C005FE79DF830
:105768003D005CE79DF83E0059E79DF83F0056E78D
:105778009DF8400053E79DF8410050E79DF842002E
:105788004DE79DF843004AE79DF8440047E79DF838
:10579800450044E79DF8460041E79DF847003EE78D
:1057A800024804F059F8002039E700BF29BC000876
:1057B80084B008B50DF1080E8EE80F009DF848304A
:1057C8001F2B74D8DFE803F01016191C1F22252898
:1057D8002B2E3134373A3D404346494C4F525558A9
:1057E8005B5E6164676A6D709DF80900BDE80840FA
:1057F80004B070479DF80B00F8E79DF80D00F5E739
:105808009DF80F00F2E79DF81100EFE79DF81300EF
:10581800ECE79DF81500E9E79DF81700E6E79DF825
:105828001900E3E79DF81B00E0E79DF81D00DDE7A0
:105838009DF81F00DAE79DF82100D7E79DF82300BF
:10584800D4E79DF82500D1E79DF82700CEE79DF81D
:105858002900CBE79DF82B00C8E79DF82D00C5E788
:105868009DF82F00C2E79DF83100BFE79DF833008F
:10587800BCE79DF83500B9E79DF83700B6E79DF815
:105888003900B3E79DF83B00B0E79DF83D00ADE770
:105898009DF83F00AAE79DF84100A7E79DF843005F
:1058A800A4E79DF84500A1E79DF847009EE7024858
:1058B80003F0D2FF002099E729BC000810B5204C5E
:1058C80000212078FFF746F960780121FFF766F894
:1058D800A0780221FFF762F8E0780321FFF75EF86D
:1058E80020790421FFF75AF860790021FFF798FA28
:1058F8000121A079FFF794FAE079FFF7E9F9207A16
:105908000021FFF783F9607A0121FFF7AFF8A07A49
:105918000221FFF7ABF8E07A0321FFF7A7F8207B15
:105928000421FFF7A3F8607B0021FFF7CDFAA07BE5
:105938000121FFF7C9FAE07BBDE81040FFF71EBA66
:10594800800E0020F0B543788FB004466C2B00F22F
:10595800D582DFE813F06D009E00B400CC00E400AF
:10596800FC0014012C01440155016D0185019D01C4
:10597800B501CD01D302E501E901ED01F101F50120
:10598800FA01FF01040209020E021302D302D30234
:10599800D30218021D0229022E02330238023D02E8
:1059A800420247024C02510256025B026002650243
:1059B8006A026F02740279027E02830288028D02F3
:1059C800920297029C02A102A602AB02B002B502A3
:1059D800D302D302D302BA02D502EB0201031703A2
:1059E8002D03430359036F0385039B03D302D3029B
:1059F800D302B103C703DD03F30309041F0435040D
:105A08006F0485049B04B104C704DD04F30409058D
:105A18001F0535054B05610577058D05A305B905F6
:105A2800CF05E5051F0635064B06610677068D0688
:105A3800BE23DA4A037013708378144693700023E8
:105A480043705370D64BD11C03F1280053F8042B34
:105A5800834241F8042BF9D11B8800220B802C23A8
:105A6800E2540133452BFBD1A578CE48A91CC9B215
:105A780002F0EBFFEB222544E870A378C7482344E3
:105A88001A71A1780531C9B20FB0BDE8F040FFF72F
:105A9800F1BA14F8030F0021FFF75CF8012322463E
:105AA80040F6B821A02002F003FA042322464FF45E
:105AB8002861A0200FB0BDE8F04002F0F9B9002538
:105AC800861C0135EDB2294616F8010FFEF766FF70
:105AD800042DF6D103342B46224640F6B921A020E6
:105AE80002F0E6F92B46224640F68421E1E700253C
:105AF800861C0135EDB2294616F8010FFEF74EFF58
:105B0800042DF6D103342B46224640F6B921A020B5
:105B180002F0CEF92B46224640F68821C9E700213B
:105B2800C078FFF77DF920790121FFF779F903346F
:105B3800A078FFF7CDF80323224640F6BD21A02028
:105B480002F0B6F90423224640F68C21B1E7002181
:105B5800C078FFF765F920790121FFF761F903346F
:105B6800A078FFF7B5F80323224640F6BD21A02010
:105B780002F09EF9042322464FF4296199E7002197
:105B8800C078FFF74DF920790121FFF749F903346F
:105B9800A078FFF79DF80323224640F6BD21A020F8
:105BA80002F086F90423224640F6942181E7002179
:105BB800C078FFF735F920790121FFF731F903346F
:105BC800A078FFF785F80323224640F6BD21A020E0
:105BD80002F06EF90423224640F6982169E714F88A
:105BE800030F0021FFF712F8012322464FF42C611E
:105BF800A02002F05DF90423224640F69C2158E7D4
:105C08000025861C0135EDB2294616F8010FFEF76E
:105C18002DFF042DF6D103342B46224640F6C12130
:105C2800A02002F045F92B4622464FF42A6140E7AE
:105C38000025861C0135EDB2294616F8010FFEF73E
:105C480015FF042DF6D103342B46224640F6C12118
:105C5800A02002F02DF92B46224640F6A42128E781
:105C68000021C078FFF730F920790121FFF72CF9DE
:105C78000334A078FFF782F80323224640F6C521B3
:105C8800A02002F015F90423224640F6A82110E7C7
:105C98000021C078FFF718F920790121FFF714F9DE
:105CA8000334A078FFF76AF80323224640F6C5219B
:105CB800A02002F0FDF80423224640F6AC21F8E6C5
:105CC8000021C078FFF700F920790121FFF7FCF8DF
:105CD8000334A078FFF752F80323224640F6C52183
:105CE800A02002F0E5F8042322464FF42B61E0E6F9
:105CF8000021C078FFF7E8F820790121FFF7E4F8E0
:105D08000334A078FFF73AF80323224640F6C5216A
:105D1800A02002F0CDF80423224640F6B421C8E6BC
:105D28004023C21C0021C4E64023C21C1946C0E619
:105D38004023C21C8021BCE64023C21CC021B8E617
:105D48004023C21C4FF48071B3E64023C21C4FF4B9
:105D5800A071AEE64023C21C4FF4C071A9E64023EF
:105D6800C21C4FF4E071A4E64023C21C4FF400713A
:105D78009FE64023C21C4FF410719AE64023C21CD0
:105D88004FF4207195E64023C21C4FF4307190E621
:105D98004023C21C4FF440718BE600BF040300206F
:105DA800D60A0020050300204023C21C4FF450717E
:105DB8007FE64023C21C4FF460717AE64023C21C80
:105DC8004FF4707175E64023C21C4FF4806170E691
:105DD8004023C21C4FF488616BE64023C21C4FF479
:105DE800906166E64023C21C4FF4986161E6402347
:105DF800C21C4FF4A0615CE64023C21C4FF4A861AA
:105E080057E64023C21C4FF4B06152E64023C21C3F
:105E18004FF4B8614DE64023C21C4FF4C06148E618
:105E28004023C21C4FF4C86143E64023C21C4FF410
:105E3800D0613EE64023C21C4FF4D86139E64023C6
:105E4800C21C4FF4E06134E64023C21C4FF4E86101
:105E58002FE64023C21C4FF4F0612AE64023C21CFF
:105E68004FF4F86125E64023C21C4FF4006120E698
:105E78004023C21C4FF404611BE64023C21C4FF4AC
:105E8800086116E64023C21C4FF40C6111E640235A
:105E9800C21C4FF410610CE64023C21C4FF414617D
:105EA80007E64023C21C4FF4186102E64023C21CD7
:105EB8004FF41C61FDE54023C21C4FF42061F8E556
:105EC8004023C21C4FF42461F3E56F46C7490C9088
:105ED800D1F800C0D1F804E08A68CB6801F1100558
:105EE80001F140043E4628686968083503C6A542A2
:105EF8003746F7D160467146FFF7C4F80FB0F0BDDA
:105F08006F46BB490C90D1F800C0D1F804E08A680C
:105F1800CB6801F1100501F140043E462868696824
:105F2800083503C6A5423746F7D1E3E76F46B149BE
:105F38000C90D1F800C0D1F804E08A68CB6801F170
:105F4800100501F140043E4628686968083503C613
:105F5800A5423746F7D1CDE76F46A7490C90D1F84F
:105F680000C0D1F804E08A68CB6801F1100501F19E
:105F780040043E4628686968083503C6A542374686
:105F8800F7D1B7E76F469D490C90D1F800C0D1F81A
:105F980004E08A68CB6801F1100501F140043E462F
:105FA80028686968083503C6A5423746F7D1A1E7CE
:105FB8006F4693490C90D1F800C0D1F804E08A6884
:105FC800CB6801F1100501F140043E462868696874
:105FD800083503C6A5423746F7D18BE76F4689498E
:105FE8000C90D1F800C0D1F804E08A68CB6801F1C0
:105FF800100501F140043E4628686968083503C663
:10600800A5423746F7D175E76F467F490C90D1F81E
:1060180000C0D1F804E08A68CB6801F1100501F1ED
:1060280040043E4628686968083503C6A5423746D5
:10603800F7D15FE76F4675490C90D1F800C0D1F8E9
:1060480004E08A68CB6801F1100501F140043E467E
:1060580028686968083503C6A5423746F7D149E775
:106068006F466B490C90D1F800C0D1F804E08A68FB
:10607800CB6801F1100501F140043E4628686968C3
:10608800083503C6A5423746F7D133E76F4661495D
:106098000C90D1F800C0D1F804E08A68CB6801F10F
:1060A800100501F140043E4628686968083503C6B2
:1060B800A5423746F7D11DE76F4657490C90D1F8EE
:1060C80000C0D1F804E08A68CB6801F1100501F13D
:1060D80040043E4628686968083503C6A542374625
:1060E800F7D107E76F464D490C90D1F800C0D1F8B9
:1060F80004E08A68CB6801F1100501F140043E46CE
:1061080028686968083503C6A5423746F7D1F1E61D
:106118006F4643490C90D1F800C0D1F804E08A6872
:10612800CB6801F1100501F140043E462868696812
:10613800083503C6A5423746F7D1DBE66F4639492D
:106148000C90D1F800C0D1F804E08A68CB6801F15E
:10615800100501F140043E4628686968083503C601
:10616800A5423746F7D1C5E66F462F490C90D1F8BE
:1061780000C0D1F804E08A68CB6801F1100501F18C
:1061880040043E4628686968083503C6A542374674
:10619800F7D1AFE66F4625490C90D1F800C0D1F889
:1061A80004E08A68CB6801F1100501F140043E461D
:1061B80028686968083503C6A5423746F7D199E6C5
:1061C8006F461B490C90D1F800C0D1F804E08A68EA
:1061D800CB6801F1100501F140043E462868696862
:1061E800083503C6A5423746F7D183E6000B0020E1
:1061F80010060020400E0020D006002010050020C8
:10620800400D0020D00E0020100A0020900A002027
:1062180050090020000E0020500A0020400C0020E9
:1062280090070020D0080020900E002010080020C1
:10623800900400206F46C5490C90D1F800C0D1F8F1
:1062480004E08A68CB6801F1100501F140043E467C
:1062580028686968083503C6A5423746F7D149E674
:106268006F46BB490C90D1F800C0D1F804E08A68A9
:10627800CB6801F1100501F140043E4628686968C1
:10628800083503C6A5423746F7D133E66F46B1490C
:106298000C90D1F800C0D1F804E08A68CB6801F10D
:1062A800100501F140043E4628686968083503C6B0
:1062B800A5423746F7D11DE66F46A7490C90D1F89D
:1062C80000C0D1F804E08A68CB6801F1100501F13B
:1062D80040043E4628686968083503C6A542374623
:1062E800F7D107E66F469D490C90D1F800C0D1F868
:1062F80004E08A68CB6801F1100501F140043E46CC
:1063080028686968083503C6A5423746F7D1F1E51C
:106318006F4693490C90D1F800C0D1F804E08A6820
:10632800CB6801F1100501F140043E462868696810
:10633800083503C6A5423746F7D1DBE56F468949DC
:106348000C90D1F800C0D1F804E08A68CB6801F15C
:10635800100501F140043E4628686968083503C6FF
:10636800A5423746F7D1C5E56F467F490C90D1F86D
:1063780000C0D1F804E08A68CB6801F1100501F18A
:1063880040043E4628686968083503C6A542374672
:10639800F7D1AFE56F4675490C90D1F800C0D1F838
:1063A80004E08A68CB6801F1100501F140043E461B
:1063B80028686968083503C6A5423746F7D199E5C4
:1063C8006F466B490C90D1F800C0D1F804E08A6898
:1063D800CB6801F1100501F140043E462868696860
:1063E800083503C6A5423746F7D183E56F466149AC
:1063F8000C90D1F800C0D1F804E08A68CB6801F1AC
:10640800100501F140043E4628686968083503C64E
:10641800A5423746F7D16DE56F4657490C90D1F83C
:1064280000C0D1F804E08A68CB6801F1100501F1D9
:1064380040043E4628686968083503C6A5423746C1
:10644800F7D157E56F464D490C90D1F800C0D1F807
:1064580004E08A68CB6801F1100501F140043E466A
:1064680028686968083503C6A5423746F7D141E56B
:106478006F4643490C90D1F800C0D1F804E08A680F
:10648800CB6801F1100501F140043E4628686968AF
:10649800083503C6A5423746F7D12BE56F4639497B
:1064A8000C90D1F800C0D1F804E08A68CB6801F1FB
:1064B800100501F140043E4628686968083503C69E
:1064C800A5423746F7D115E56F462F490C90D1F80C
:1064D80000C0D1F804E08A68CB6801F1100501F129
:1064E80040043E4628686968083503C6A542374611
:1064F800F7D1FFE46F4625490C90D1F800C0D1F8D8
:1065080004E08A68CB6801F1100501F140043E46B9
:1065180028686968083503C6A5423746F7D1E9E413
:106528006F461B490C90D1F800C0D1F804E08A6886
:10653800CB6801F1100501F140043E4628686968FE
:10654800083503C6A5423746F7D1D3E4C00B00206F
:10655800800B002050050020C00C0020D007002030
:1065680010070020400B002050040020800D002060
:10657800100900209005002090060020D00400207B
:1065880050060020000D0020500700209008002031
:10659800D00500206F4641490C90D1F800C0D1F8D1
:1065A80004E08A68CB6801F1100501F140043E4619
:1065B80028686968083503C6A5423746F7D199E4C3
:1065C8006F4637490C90D1F800C0D1F804E08A68CA
:1065D800CB6801F1100501F140043E46286869685E
:1065E800083503C6A5423746F7D183E46F462D49DF
:1065F8000C90D1F800C0D1F804E08A68CB6801F1AA
:10660800100501F140043E4628686968083503C64C
:10661800A5423746F7D16DE46F4623490C90D1F86F
:1066280000C0D1F804E08A68CB6801F1100501F1D7
:1066380040043E4628686968083503C6A5423746BF
:10664800F7D157E46F4619490C90D1F800C0D1F83A
:1066580004E08A68CB6801F1100501F140043E4668
:1066680028686968083503C6A5423746F7D141E46A
:106678006F460F490C90D1F800C0D1F804E08A6841
:10668800CB6801F1100501F140043E4628686968AD
:10669800083503C6A5423746F7D12BE490090020F8
:1066A800D009002050080020800C0020C00D0020D8
:1066B800000C00202DE9F0410446A8B0457864227A
:1066C80000210FA802F0EBFB237828AA8DF83C30B4
:1066D800A3788DF83D508DF83E301A4423441B7939
:1066E80002F8603C6C2D01F2AB83DFE815F06D0019
:1066F80080009E0012017B01F10144029702EA0228
:1067080003038F03F7034A049D041305A90B6605C9
:106718007C059205A805BE05D405EA0500061606FF
:106728002C064206A90BA90BA90B58066E0684066F
:106738009A06D706ED06030719072F0745075B07D3
:10674800710787079D07B307C907DF07F5070B0818
:10675800210837084D0863089F08B508CB08E108E9
:10676800F7080D0923093909A90BA90BA90B4F092A
:106778005C0969097609830990099D09AA09B7097D
:10678800C409D109A90BA90BA90BDE09EB09F80962
:10679800050A120A1F0A2C0A390A460A8B0A980A9D
:1067A800A50AB20ABF0ACC0AD90AE60AF30A000BFC
:1067B8000D0B1A0B270B340B410B4E0B5B0B680BA5
:1067C800750B820B8F0B9C0BB24B0DF13F0203F143
:1067D800280153F8040B8B4242F8040BF9D11B88AB
:1067E80013800FA8FFF7AEF828B0BDE8F081EE4699
:1067F800E278A94BA94D9A71E37805F110060C933C
:10680800D5F80080D5F804C0AA68EB68403577460B
:1068180030687168083603C7AE42BE46F7D14046B5
:106828006146FEF75DFCE0706CE0EE46D4F80320AC
:10683800994B9B4DC3F80720E37805F110060C939C
:10684800D5F80080D5F804C0AA68EB6840357746CB
:1068580030687168083603C7AE42BE46F7D1404675
:106868006146FEF745FDEE4623798E4DE0700C93A8
:10687800D5F80080D5F804C0AA68EB6805F11006C1
:106888004035774630687168083603C7AE42BE4661
:10689800F7D140466146FEF72BFDEE466379824DFF
:1068A80020710C93D5F80080D5F804C0AA68EB686D
:1068B80005F110064035774630687168083603C719
:1068C800AE42BE46F7D140466146FEF711FDEE46A0
:1068D800A379764D60710C93D5F80080D5F804C083
:1068E800AA68EB6805F1100640357746306871688C
:1068F800083603C7AE42BE46F7D140466146FEF7AA
:10690800F7FCA071A278214605320FA802F0BCFA64
:1069180067E7EE46D4F803205F4B654DC3F80B20BC
:10692800E37805F110060C93D5F80080D5F804C07B
:10693800AA68EB684035774630687168083603C73F
:10694800AE42BE46F7D140466146FEF7D1FCEE4660
:106958002379584DE0700C93D5F80080D5F804C021
:10696800AA68EB6805F1100640357746306871680B
:10697800083603C7AE42BE46F7D140466146FEF729
:10698800B7FCEE4663794C4D20710C93D5F8008026
:10699800D5F804C0AA68EB6805F1100640357746BB
:1069A80030687168083603C7AE42BE46F7D1404624
:1069B8006146FEF79DFCEE46A379404D60710C934D
:1069C800D5F80080D5F804C0AA68EB6805F1100670
:1069D8004035774630687168083603C7AE42BE4610
:1069E800F7D18AE72346EE4633F8031F344A354D7C
:1069F80011809B7805F110069370E37840350C936D
:106A080055F8408C55F83CCC55F8382C55F8343CA2
:106A1800774630687168083603C7AE42BE46F7D17C
:106A280040466146FEF7C4FEEE462379264DE070E7
:106A38000C93D5F80080D5F804C0AA68EB6805F176
:106A480010064035774630687168083603C7AE428D
:106A5800BE46F7D140466146FEF7AAFEEE46637988
:106A68001A4D20710C93D5F80080D5F804C0AA6897
:106A7800EB6805F1100640357746306871680836CE
:106A880003C7AE42BE46F7D140466146FEF798FDC1
:106A9800607137E7D60A0020D00A0020000B0020DA
:106AA80010060020400E0020D0060020100500200F
:106AB800400D0020D00E0020100A0020900A00206F
:106AC800DF0A002050090020000E0020500A002094
:106AD8002346EE4633F8031FBA4ABB4D11809B7814
:106AE80005F110069370E37840350C9355F8408C07
:106AF80055F83CCC55F8382C55F8343C7746306876
:106B08007168083603C7AE42BE46F7D140466146B3
:106B1800FEF74EFEEE462379AC4DE0700C93D5F8A7
:106B28000080D5F804C0AA68EB6805F11006403566
:106B3800774630687168083603C7AE42BE46F7D15B
:106B480040466146FEF734FEEE466379A04D20715B
:106B58000C93D5F80080D5F804C0AA68EB6805F155
:106B680010064035774630687168083603C7AE426C
:106B7800BE46F7D188E72346EE4633F8031F954A09
:106B8800954D11809B7805F110069370E378403598
:106B98000C9355F8408C55F83CCC55F8382C55F8E2
:106BA800343C774630687168083603C7AE42BE4643
:106BB800F7D140466146FEF7FBFDEE462379874D47
:106BC800E0700C93D5F80080D5F804C0AA68EB688B
:106BD80005F110064035774630687168083603C7F6
:106BE800AE42BE46F7D140466146FEF7E1FDEE46AD
:106BF80063797B4D20710C93D5F80080D5F804C0DB
:106C0800AA68EB6805F11006403577463068716868
:106C1800083603C7AE42BE46F7D135E72346EE46EF
:106C280033F8031F6F4A704D11809B7805F11006E9
:106C38009370E37840350C9355F8408C55F83CCC6C
:106C480055F8382C55F8343C774630687168083662
:106C580003C7AE42BE46F7D140466146FEF7A8FDDF
:106C6800EE462379614DE0700C93D5F80080D5F895
:106C780004C0AA68EB6805F110064035774630680D
:106C88007168083603C7AE42BE46F7D14046614632
:106C9800FEF78EFDEE466379554D20710C93D5F8BD
:106CA8000080D5F804C0AA68EB6805F110064035E5
:106CB800774630687168083603C7AE42BE46F7D1DA
:106CC800E2E6EE46E2784B4B4B4DDA76E37805F197
:106CD80010060C93D5F80080D5F804C0AA68EB68B4
:106CE8004035774630687168083603C7AE42BE46FD
:106CF800F7D194E5EE46D4F803203E4B3F4DDA61D8
:106D0800E37805F110060C93D5F80080D5F804C097
:106D1800AA68EB684035774630687168083603C75B
:106D2800AE42BE46F7D140466146FEF7E1FAEE466E
:106D38002379334DE0700C93D5F80080D5F804C062
:106D4800AA68EB6805F11006403577463068716827
:106D5800083603C7AE42BE46F7D140466146FEF745
:106D6800C7FAEE466379274D20710C93D5F8008059
:106D7800D5F804C0AA68EB6805F1100640357746D7
:106D880030687168083603C7AE42BE46F7D1404640
:106D98006146FEF7ADFAEE46A3791B4D60710C9380
:106DA800D5F80080D5F804C0AA68EB6805F110068C
:106DB8004035774630687168083603C7AE42BE462C
:106DC800F7D19AE5E20A0020400C00209007002045
:106DD800D0080020E50A0020900E002010080020AE
:106DE80090040020E80A0020C00B0020800B00203F
:106DF80050050020D00A0020C00C0020D007002039
:106E080010070020400B002050040020EE46D4F864
:106E18000320AF4BAF4D1A62E37805F110060C93CF
:106E2800D5F80080D5F804C0AA68EB6840357746E5
:106E380030687168083603C7AE42BE46F7D140468F
:106E48006146FEF755FAEE462379A34DE0700C93A0
:106E5800D5F80080D5F804C0AA68EB6805F11006DB
:106E68004035774630687168083603C7AE42BE467B
:106E7800F7D140466146FEF73BFAEE466379974DF7
:106E880020710C93D5F80080D5F804C0AA68EB6887
:106E980005F110064035774630687168083603C733
:106EA800AE42BE46F7D140466146FEF721FAEE46AD
:106EB800A3798B4D60710C93D5F80080D5F804C088
:106EC800AA68EB6805F110064035774630687168A6
:106ED800083603C7AE42BE46F7D10EE52346EE4656
:106EE80033F8031F7F4A804D11809B7805F1100607
:106EF8009370E37840350C9355F8408C55F83CCCAA
:106F080055F8382C55F8343C77463068716808369F
:106F180003C7AE42BE46F7D140466146FEF748FC7D
:106F2800EE462379714DE0700C93D5F80080D5F8C2
:106F380004C0AA68EB6805F110064035774630684A
:106F48007168083603C7AE42BE46F7D1404661466F
:106F5800FEF72EFCEE466379654D20710C93D5F84B
:106F68000080D5F804C0AA68EB6805F11006403522
:106F7800774630687168083603C7AE42BE46F7D117
:106F880082E52346EE4633F8031F5A4A5A4D1180CC
:106F98009B7805F110069370E37840350C9355F80B
:106FA800408C55F83CCC55F8382C55F8343C77468D
:106FB80030687168083603C7AE42BE46F7D140460E
:106FC8006146FEF7F5FBEE4623794C4DE0700C93D5
:106FD800D5F80080D5F804C0AA68EB6805F110065A
:106FE8004035774630687168083603C7AE42BE46FA
:106FF800F7D140466146FEF7DBFBEE466379404D2C
:1070080020710C93D5F80080D5F804C0AA68EB6805
:1070180005F110064035774630687168083603C7B1
:10702800AE42BE46F7D12FE52346EE4633F8031F9E
:10703800344A354D11809B7805F110069370E3783A
:1070480040350C9355F8408C55F83CCC55F8382C05
:1070580055F8343C774630687168083603C7AE4245
:10706800BE46F7D140466146FEF7A2FBEE462379BD
:10707800264DE0700C93D5F80080D5F804C0AA68B6
:10708800EB6805F1100640357746306871680836B8
:1070980003C7AE42BE46F7D140466146FEF788FBBD
:1070A800EE4663791A4D20710C93D5F80080D5F817
:1070B80004C0AA68EB6805F11006403577463068C9
:1070C8007168083603C7AE42BE46F7D1DCE400BF9C
:1070D800D00A0020800D0020100900209005002013
:1070E80090060020F40A0020D0040020500600205A
:1070F800000D0020F70A002050070020900800200B
:10710800D0050020FA0A002090090020D0090020AC
:10711800500800202346EE4633F8031FCC4ACD4DD5
:1071280011809B7805F110069370E37840350C9335
:1071380055F8408C55F83CCC55F8382C55F8343C6B
:10714800774630687168083603C7AE42BE46F7D145
:1071580040466146FEF72CFBEE462379BE4DE070B3
:107168000C93D5F80080D5F804C0AA68EB6805F13F
:1071780010064035774630687168083603C7AE4256
:10718800BE46F7D140466146FEF712FBEE466379EC
:10719800B24D20710C93D5F80080D5F804C0AA68C8
:1071A800EB6805F110064035774630687168083697
:1071B80003C7AE42BE46F7D166E4A94AE31C43348E
:1071C80053F8041BA34242F8041BF9D1A44B0DF158
:1071D8003F0203F1400153F8040B8B4242F8040BC1
:1071E800F9D1FFF7FEBA9F4AE31C433453F8041B56
:1071F800A34242F8041BF9D19A4B0DF13F0203F167
:10720800400153F8040B8B4242F8040BF9D1FFF705
:10721800E8BA954AE31C433453F8041BA34242F8E6
:10722800041BF9D1904B0DF13F0203F1400153F8D3
:10723800040B8B4242F8040BF9D1FFF7D2BA8B4A00
:10724800E31C433453F8041BA34242F8041BF9D14E
:10725800864B0DF13F0203F1400153F8040B8B42BA
:1072680042F8040BF9D1FFF7BCBA814AE31C433456
:1072780053F8041BA34242F8041BF9D17C4B0DF1CF
:107288003F0203F1400153F8040B8B4242F8040B10
:10729800F9D1FFF7A6BA774AE31C433453F8041B25
:1072A800A34242F8041BF9D1724B0DF13F0203F1DE
:1072B800400153F8040B8B4242F8040BF9D1FFF755
:1072C80090BA6D4AE31C433453F8041BA34242F8B6
:1072D800041BF9D1684B0DF13F0203F1400153F84B
:1072E800040B8B4242F8040BF9D1FFF77ABA634AD0
:1072F800E31C433453F8041BA34242F8041BF9D19E
:107308005E4B0DF13F0203F1400153F8040B8B4231
:1073180042F8040BF9D1FFF764BA594AE31C433425
:1073280053F8041BA34242F8041BF9D1544B0DF146
:107338003F0203F1400153F8040B8B4242F8040B5F
:10734800F9D1FFF74EBA4F4AE31C433453F8041BF4
:10735800A34242F8041BF9D14A4B0DF13F0203F155
:10736800400153F8040B8B4242F8040BF9D1FFF7A4
:1073780038BA454AE31C433453F8041BA34242F885
:10738800041BF9D1404B0DF13F0203F1400153F8C2
:10739800040B8B4242F8040BF9D1FFF722BA3B4A9F
:1073A800E31C433453F8041BA34242F8041BF9D1ED
:1073B800364B0DF13F0203F1400153F8040B8B42A9
:1073C80042F8040BF9D1FFF70CBA314AE31C4334F5
:1073D80053F8041BA34242F8041BF9D12C4B0DF1BE
:1073E8003F0203F1400153F8040B8B4242F8040BAF
:1073F800F9D1FFF7F6B9274AE31C433453F8041BC5
:10740800A34242F8041BF9D1224B0DF13F0203F1CC
:10741800400153F8040B8B4242F8040BF9D1FFF7F3
:10742800E0B91D4AE31C433453F8041BA34242F855
:10743800041BF9D1184B0DF13F0203F1400153F839
:10744800040B8B4242F8040BF9D1FFF7CAB900BF0D
:10745800FD0A0020800C0020C00D0020000C002038
:10746800000B002010060020400E0020D00600204F
:1074780010050020400D0020D00E0020100A00202A
:10748800900A002050090020000E0020500A002019
:10749800400C002090070020D0080020D04AE31CB0
:1074A800433453F8041BA34242F8041BF9D1CC4BD4
:1074B8000DF13F0203F1400153F8040B8B4242F8EF
:1074C800040BF9D1FFF78DB9C64AE31C433453F8CE
:1074D800041BA34242F8041BF9D1C24B0DF13F0231
:1074E80003F1400153F8040B8B4242F8040BF9D125
:1074F800FFF777B9BC4AE31C433453F8041BA34293
:1075080042F8041BF9D1B84B0DF13F0203F14001D9
:1075180053F8040B8B4242F8040BF9D1FFF761B919
:10752800B24AE31C433453F8041BA34242F8041B39
:10753800F9D1AE4B0DF13F0203F1400153F8040BB2
:107548008B4242F8040BF9D1FFF74BB9A84AE31C68
:10755800433453F8041BA34242F8041BF9D1A44B4B
:107568000DF13F0203F1400153F8040B8B4242F83E
:10757800040BF9D1FFF735B99E4AE31C433453F89D
:10758800041BA34242F8041BF9D19A4B0DF13F02A8
:1075980003F1400153F8040B8B4242F8040BF9D174
:1075A800FFF71FB9944AE31C433453F8041BA34262
:1075B80042F8041BF9D1904B0DF13F0203F1400151
:1075C80053F8040B8B4242F8040BF9D1FFF709B9C1
:1075D8008A4AE31C433453F8041BA34242F8041BB1
:1075E800F9D1864B0DF13F0203F1400153F8040B2A
:1075F8008B4242F8040BF9D1FFF7F3B8804AE31C39
:10760800433453F8041BA34242F8041BF9D17C4BC2
:107618000DF13F0203F1400153F8040B8B4242F88D
:10762800040BF9D1FFF7DDB8764AE31C433453F86D
:10763800041BA34242F8041BF9D1724B0DF13F021F
:1076480003F1400153F8040B8B4242F8040BF9D1C3
:10765800FFF7C7B86C4AE31C433453F8041BA34232
:1076680042F8041BF9D1684B0DF13F0203F14001C8
:1076780053F8040B8B4242F8040BF9D1FFF7B1B869
:10768800624AE31C433453F8041BA34242F8041B28
:10769800F9D15E4B0DF13F0203F1400153F8040BA1
:1076A8008B4242F8040BF9D1FFF79BB8584AE31C08
:1076B800433453F8041BA34242F8041BF9D1544B3A
:1076C8000DF13F0203F1400153F8040B8B4242F8DD
:1076D800040BF9D1FFF785B84E4AE31C433453F83D
:1076E800041BA34242F8041BF9D14A4B0DF13F0297
:1076F80003F1400153F8040B8B4242F8040BF9D113
:10770800FFF76FB8444AE31C433453F8041BA34201
:1077180042F8041BF9D1404B0DF13F0203F140013F
:1077280053F8040B8B4242F8040BF9D1FFF759B810
:107738003A4AE31C433453F8041BA34242F8041B9F
:10774800F9D1364B0DF13F0203F1400153F8040B18
:107758008B4242F8040BF9D1FFF743B8304AE31CD7
:10776800433453F8041BA34242F8041BF9D12C4BB1
:107778000DF13F0203F1400153F8040B8B4242F82C
:10778800040BF9D1FFF72DB8264AE31C433453F80C
:10779800041BA34242F8041BF9D1224B0DF13F020E
:1077A80003F1400153F8040B8B4242F8040BF9D162
:1077B800FFF717B81C4AE31C433453F8041BA342D1
:1077C80042F8041BF9D1184B0DF13F0203F14001B7
:1077D80053F8040B8B4242F8040BF9D1FFF701B8B8
:1077E800900E00201008002090040020C00B0020FC
:1077F800800B002050050020C00C0020D00700207E
:1078080010070020400B002050040020800D0020AD
:10781800100900209005002090060020D0040020C8
:1078280050060020000D002050070020D94AE31C14
:10783800433453F8041BA34242F8041BF9D1D54B37
:107848000DF13F0203F1400153F8040B8B4242F85B
:10785800040BF9D1FEF7C5BFCF4AE31C433453F8F4
:10786800041BA34242F8041BF9D1CB4B0DF13F0294
:1078780003F1400153F8040B8B4242F8040BF9D191
:10788800FEF7AFBFC54AE31C433453F8041BA342B9
:1078980042F8041BF9D1C14B0DF13F0203F140013D
:1078A80053F8040B8B4242F8040BF9D1FEF799BF49
:1078B800BB4AE31C433453F8041BA34242F8041B9D
:1078C800F9D1B74B0DF13F0203F1400153F8040B16
:1078D8008B4242F8040BF9D1FEF783BFB14AE31C8F
:1078E800433453F8041BA34242F8041BF9D1AD4BAF
:1078F8000DF13F0203F1400153F8040B8B4242F8AB
:10790800040BF9D1FEF76DBFA74AE31C433453F8C3
:10791800041BA34242F8041BF9D1A34B0DF13F020B
:1079280003F1400153F8040B8B4242F8040BF9D1E0
:10793800FEF757BF9D4AE31C433453F8041BA34288
:1079480042F8041BF9D1994B0DF13F0203F14001B4
:1079580053F8040B8B4242F8040BF9D1FEF741BFF0
:10796800934AE31C433453F8041BA34242F8041B14
:10797800F9D18F4B0DF13F0203F1400153F8040B8D
:107988008B4242F8040BF9D1FEF72BBF894B0DF15E
:107998003F0203F1400153F8040B8B4242F8040BF9
:1079A800F9D1FEF71EBF844B0DF13F0203F14001F0
:1079B80053F8040B8B4242F8040BF9D1FEF711BFC0
:1079C8007E4B0DF13F0203F1400153F8040B8B424B
:1079D80042F8040BF9D1FEF704BF794B0DF13F02D1
:1079E80003F1400153F8040B8B4242F8040BF9D120
:1079F800FEF7F7BE734B0DF13F0203F1400153F858
:107A0800040B8B4242F8040BF9D1FEF7EABE6E4B29
:107A18000DF13F0203F1400153F8040B8B4242F889
:107A2800040BF9D1FEF7DDBE684B0DF13F0203F1FF
:107A3800400153F8040B8B4242F8040BF9D1FEF7CE
:107A4800D0BE634B0DF13F0203F1400153F8040B24
:107A58008B4242F8040BF9D1FEF7C3BE5D4B0DF122
:107A68003F0203F1400153F8040B8B4242F8040B28
:107A7800F9D1FEF7B6BE584B0DF13F0203F14001B4
:107A880053F8040B8B4242F8040BF9D1FEF7A9BE58
:107A9800524B0DF13F0203F1400153F8040B8B42A6
:107AA80042F8040BF9D1FEF79CBE4D4B0DF13F0295
:107AB80003F1400153F8040B8B4242F8040BF9D14F
:107AC800FEF78FBE474B0DF13F0203F1400153F81B
:107AD800040B8B4242F8040BF9D1FEF782BE424BED
:107AE8000DF13F0203F1400153F8040B8B4242F8B9
:107AF800040BF9D1FEF775BE3C4B0DF13F0203F1C3
:107B0800400153F8040B8B4242F8040BF9D1FEF7FD
:107B180068BE374B0DF13F0203F1400153F8040BE7
:107B28008B4242F8040BF9D1FEF75BBE314B0DF1E5
:107B38003F0203F1400153F8040B8B4242F8040B57
:107B4800F9D1FEF74EBE2C4B0DF13F0203F1400177
:107B580053F8040B8B4242F8040BF9D1FEF741BEEF
:107B6800264B0DF13F0203F1400153F8040B8B4201
:107B780042F8040BF9D1FEF734BE214B0DF13F0258
:107B880003F1400153F8040B8B4242F8040BF9D17E
:107B9800FEF727BE90080020D0050020900900209D
:107BA800D009002050080020800C0020C00D0020C3
:107BB800000C0020000B002010060020400E0020C2
:107BC800D006002010050020400D0020D00E002017
:107BD800100A0020900A002050090020000E002002
:107BE800500A0020400C002090070020D0080020F8
:107BF800900E00201008002090040020C00B0020E8
:107C0800800B0020924B0DF13F0203F1400153F825
:107C1800040B8B4242F8040BF9D1FEF7E2BD8D4B01
:107C28000DF13F0203F1400153F8040B8B4242F877
:107C3800040BF9D1FEF7D5BD874B0DF13F0203F1D7
:107C4800400153F8040B8B4242F8040BF9D1FEF7BC
:107C5800C8BD824B0DF13F0203F1400153F8040BFC
:107C68008B4242F8040BF9D1FEF7BBBD7C4B0DF1FA
:107C78003F0203F1400153F8040B8B4242F8040B16
:107C8800F9D1FEF7AEBD774B0DF13F0203F140018C
:107C980053F8040B8B4242F8040BF9D1FEF7A1BD4F
:107CA800714B0DF13F0203F1400153F8040B8B4275
:107CB80042F8040BF9D1FEF794BD6C4B0DF13F026D
:107CC80003F1400153F8040B8B4242F8040BF9D13D
:107CD800FEF787BD664B0DF13F0203F1400153F8F3
:107CE800040B8B4242F8040BF9D1FEF77ABD614BC5
:107CF8000DF13F0203F1400153F8040B8B4242F8A7
:107D0800040BF9D1FEF76DBD5B4B0DF13F0203F19A
:107D1800400153F8040B8B4242F8040BF9D1FEF7EB
:107D280060BD564B0DF13F0203F1400153F8040BBF
:107D38008B4242F8040BF9D1FEF753BD504B0DF1BD
:107D48003F0203F1400153F8040B8B4242F8040B45
:107D5800F9D1FEF746BD4B4B0DF13F0203F140014F
:107D680053F8040B8B4242F8040BF9D1FEF739BDE6
:107D7800454B0DF13F0203F1400153F8040B8B42D0
:107D880042F8040BF9D1FEF72CBD404B0DF13F0230
:107D980003F1400153F8040B8B4242F8040BF9D16C
:107DA800FEF71FBD3A4B0DF13F0203F1400153F8B6
:107DB800040B8B4242F8040BF9D1FEF712BD354B88
:107DC8000DF13F0203F1400153F8040B8B4242F8D6
:107DD800040BF9D1FEF705BD2F4B0DF13F0203F15E
:107DE800400153F8040B8B4242F8040BF9D1FEF71B
:107DF800F8BC2A4B0DF13F0203F1400153F8040B84
:107E08008B4242F8040BF9D1FEF7EBBC244B0DF181
:107E18003F0203F1400153F8040B8B4242F8040B74
:107E2800F9D1FEF7DEBC1F4B0DF13F0203F1400113
:107E380053F8040B8B4242F8040BF9D1FEF7D1BC7E
:107E480040F2CD721849194801F092FCFEF7C9BCFE
:107E580050050020C00C0020D0070020100700208B
:107E6800400B002050040020800D00201009002045
:107E78009005002090060020D00400205006002025
:107E8800000D00205007002090080020D005002099
:107E980090090020D009002050080020800C002004
:107EA800C00D0020000C002060BC000839BC000890
:107EB8001FB50A248DE81C000A4610230146054810
:107EC800F9F720FF04460520F9F78EF9204604B09B
:107ED80010BD00BF100F00201FB50A248DE81C003C
:107EE8000A46102301460548F9F79CFF0446052079
:107EF800F9F77AF9204604B010BD00BF100F002032
:107F080010B54023DF4A0021A020FFF7E5FF4023FA
:107F1800DD4A1946A020FFF7DFFF4023DB4A802116
:107F2800A020FFF7D9FF4023D94AC021A020FFF79E
:107F3800D3FF4023D74A4FF48071A020FFF7CCFF2E
:107F48004023D54A4FF4A071A020FFF7C5FF402376
:107F5800D24A4FF4C071A020FFF7BEFF4023D04A99
:107F68004FF4E071A020FFF7B7FF4023CD4A4FF44C
:107F78000071A020FFF7B0FF4023CB4A4FF41071E7
:107F8800A020FFF7A9FF4023C84A4FF42071A02082
:107F9800FFF7A2FF4023C64A4FF43071A020FFF735
:107FA8009BFF4023C34A4FF44071A020FFF794FF82
:107FB8004023C14A4FF45071A020FFF78DFF4023A2
:107FC800BE4A4FF46071A020FFF786FF4023BC4AE9
:107FD8004FF47071A020FFF77FFF4023B94A4FF498
:107FE8008061A020FFF778FF4023B74A4FF48861EB
:107FF800A020FFF771FF4023B44A4FF49061A020FE
:10800800FFF76AFF4023B24A4FF49861A020FFF7B8
:1080180063FF4023AF4A4FF4A061A020FFF75CFF45
:108028004023AD4A4FF4A861A020FFF755FF402335
:10803800AA4A4FF4B061A020FFF74EFF4023A84A98
:108048004FF4B861A020FFF747FF4023A54A4FF43B
:10805800C061A020FFF740FF4023A34A4FF4C86146
:10806800A020FFF739FF4023A04A4FF4D061A02099
:10807800FFF732FF40239E4A4FF4D861A020FFF754
:108088002BFF40239B4A4FF4E061A020FFF724FF19
:108098004023994A4FF4E861A020FFF71DFF4023D1
:1080A800964A4FF4F061A020FFF716FF4023944A48
:1080B8004FF4F861A020FFF70FFF4023914A4FF4D7
:1080C8000061A020FFF708FF40238F4A4FF40461A6
:1080D800A020FFF701FF40238C4A4FF40861A0203D
:1080E800FFF7FAFE40238A4A4FF40C61A020FFF7FD
:1080F800F3FE4023874A4FF41061A020FFF7ECFEFF
:108108004023854A4FF41461A020FFF7E5FE402381
:10811800824A4FF41861A020FFF7DEFE4023804A10
:108128004FF41C61A0207F4CFFF7D6FE40237E4A07
:108138004FF42061A020FFF7CFFE40237B4A4FF485
:108148002461A020FFF7C8FE224601234FF42861CE
:10815800A020FFF7C1FE621C042340F68421A02062
:10816800FFF7BAFE621D042340F68821A020FFF71E
:10817800B3FE04F10902032340F68C21A020FFF787
:10818800ABFE04F10C0203234FF42961A020FFF792
:10819800A3FE04F10F02032340F69421A020FFF769
:1081A8009BFE04F11202032340F69821A020FFF75A
:1081B80093FE04F11502012340F69C21A020FFF74D
:1081C8008BFE04F1160204234FF42A61A020FFF766
:1081D80083FE04F11A02042340F6A421A020FFF72D
:1081E8007BFE04F11E02032340F6A821A020FFF71E
:1081F80073FE04F12102032340F6AC21A020FFF70F
:108208006BFE04F1240203234FF42B61A020FFF737
:1082180063FE04F12702464C032340F6B421A02054
:10822800FFF75AFE2246012340F6B821A020FFF7A7
:1082380053FE621C042340F6B921A020FFF74CFE30
:10824800621D032340F6BD21A020FFF745FE04F17F
:10825800080201234FF42C61A020FFF73DFE04F132
:108268000902042340F6C121A020FFF735FE04F1DE
:108278000D020323BDE8104040F6C521A020FFF7FA
:108288002BBE00BF000B002010060020400E00206F
:10829800D006002010050020400D0020D00E002040
:1082A800100A0020900A002050090020000E00202B
:1082B800500A0020400C002090070020D008002021
:1082C800900E00201008002090040020C00B002011
:1082D800800B002050050020C00C0020D007002093
:1082E80010070020400B002050040020800D0020C3
:1082F800100900209005002090060020D0040020DE
:1083080050060020000D0020500700209008002093
:10831800D005002090090020D00900205008002036
:10832800800C0020D60A0020C00D0020000C002080
:10833800800E002010B514460A230248FAF740FBC5
:10834800204610BDC80F002008B502680B4B9A42A2
:1083580012D10B4A1368013313600A4A13680133B8
:108368001360094B1B783BB1FBF768F9132881BFF1
:10837800064A13680133136008BD00BF00100040AF
:10838800D4030020D0030020D8030020CC03002011
:1083980002680E4B9A4217D10D490E4A0978137894
:1083A8000D48EB29C15404BF01200C4903F1010316
:1083B800DBB208BF0870632B88BF00230449137021
:1083C80007480122FAF792BB704700BF00480040F7
:1083D800081000206D1000206E100020C40F00202F
:1083E800C80F0020B0F5807F10B5014607D1294B92
:1083F8001A787AB9012228490A701A701AE0B0F579
:10840800805F0CD1234B1A7822B90221224A1170BD
:108418000122F2E7002221491A700A6010BDB0F566
:10842800005F18D11B4C2378EBB903221A4B1A7042
:10843800012323701A4A1B4912684CF25033B2FBCD
:10844800F1F253431A46013B002AFBD1124B18782C
:10845800FBF798FB10BDB0F5804F0ED10D4C23787B
:108468000BB90422E2E71048F9F7BAF90128E1D17B
:1084780000230A4A2370136010BDB0F5004FD9D10C
:10848800044B1A780AB90521C0E700221A70034B79
:108498001A6010BDD80300203D040020CC03002042
:1084A8000800002040420F000004024010B592B0BE
:1084B8003022002106A800F0F2FC1422002101A8B5
:1084C80000F0EDFC0123099310230A930D230E936A
:1084D800C32302240F93042306A8119306940C9433
:1084E8001094F9F7ABFD0F230193002303934FF486
:1084F800A05304934FF48053032101A802940593D9
:10850800F9F76CFF12B010BD2DE9F04F0024ABB0A5
:108518000CAE6422002111A8BA4D00F0C0FCF8F797
:1085280037FEFFF7C3FF14220021304600F0B7FCE6
:1085380004942B6B224643F010032B632B6B47F6F6
:108548003D7103F010030493049B05942B6BAE4814
:1085580043F004032B632B6B012703F004030593FB
:10856800059B06942B6BDFF8DC8243F020032B631A
:108578002B6B4FF00C0903F020030693069B07941E
:108588002B6B43F080032B632B6B03F08003079363
:10859800079B08942B6B43F001032B632B6B03F0B1
:1085A80001030893089B09942B6B43F002032B6388
:1085B8002B6B03F002030993099B0A942B6B43F07E
:1085C80008032B632B6B03F008030A930A9B0B9495
:1085D8002B6B43F040032B632B6B03F040030B938F
:1085E8000B9BF9F703F922464DF630418748F9F716
:1085F800FDF822464EF607018548F9F7F7F82246B6
:108608004FF40F618348F9F7F1F8224640F2E1216F
:108618008148F9F7EBF822464FF6CF017F48F9F782
:10862800E5F8224647F6FC217D48F9F7DFF847F6DA
:108638003D73314674480C930E940F940D97F8F7D8
:10864800EDFF4DF63043314670480C930E940F946D
:108658000D97F8F7E3FF4EF6070331466C480C9385
:108668000E940F940D97F8F7D9FF4FF4E073314645
:1086780067480C930D940E94F8F7D0FF0E233146FB
:1086880062480C930D940E94F8F7C8FF4FF40F63EB
:10869800314660480C930E940F940D97F8F7BEFF7F
:1086A80040F2E12331465C480C930E940F940D97E9
:1086B800F8F7B4FF4FF47043314657480C93CDF8A0
:1086C80034800E97F8F7AAFF4FF480733146534869
:1086D8000C93CDF834800E97F8F7A0FF4FF6CF0330
:1086E80031464E480C930E940F940D97F8F796FF69
:1086F80047F6FC2331464A480C930E940F940D9785
:10870800F8F78CFF03942B6BDFF83C8143F40013DC
:108718002B632B6B434A03F400130393039B41F22F
:108728006F7388E80C0009234046C8F80C300C9495
:108738007460C8F80840C8F81840FAF73BF83146A2
:1087480040460C940D94FAF74FF837483749384BA0
:10875800846080E80A004FF48043C4600361446188
:108768008461C4610462F9F729FA4FF4E133314DA9
:108778003148AC6085E809002846EC602C61AC61A2
:10878800EC61C5F81490FAF7EDF822462146484600
:10879800F8F750FD4846F8F781FD224621460F209C
:1087A800F8F748FD0F20F8F779FD224621462720E3
:1087B800F8F740FD2720F8F771FD224621463620BC
:1087C800F8F738FD3620F8F769FD224621462820BB
:1087D800F8F730FD2820F8F761FD224621461720DA
:1087E800F8F728FD1720F8F759FD4046F9F7C6FEB7
:1087F8003A4612492846FAF779F9114800F0EAFA98
:1088080024E000BF00380240001002400008024087
:10881800001402400000024000040240000C024024
:108828000018024000100040100F0020005C0040BB
:10883800801A0600C80F00200048004008100020D9
:108848001811002000003110D41000206C4B214674
:108858001B68986801F008F8FFF752FBFAF764FC08
:108868002046FBF78FF9674B11AC03F14005224610
:1088780018685968083303C2AB421446F7D1624DF1
:10888800FDF71CF8A946DFF8BC816049604A0B78FF
:1088980012789A4212D000245E4A5F4F14603A78E8
:1088A800D2B2501CC0B238705C48C75C0133DBB22E
:1088B8005B48632B875494BF0B700C702B78012B8B
:1088C80032D1544B1B68642B2ED9DFF854A1524F78
:1088D8009AF802100AF101000AEB01030231DA7872
:1088E800C9B200F0CDF85446002873D14D4B3A7800
:1088F80000F1010BC0B2904264D34B4800F0ACFFCA
:108908009AF8022049481444E178053200F030FF13
:1089180064220021424800F0C2FA0020387089F829
:108928000000FAF779FAB0E7FAF77CFA0128CCD018
:108938003F4C2368B3F5FA7F0CD94FF400513D48FA
:10894800F8F74EFF002852D13B4B1878FBF71AF97D
:1089580000232360394C2368B3F5FA7F95D9304654
:10896800FCF706FB96E80300FCF736FBBE238DF800
:1089780044306D238DF84530082330688DF8463033
:10898800B388CDF847000A210DF14500ADF84B300A
:1089980000F05BF89DF846302AAA1344EB228DF8C4
:1089A8004F0003F8602C9DF8461011A80531C9B294
:1089B800FCF760FB4FF400414046F8F71CFF00232A
:1089C800236062E7215C1846019300F0D1FE584607
:1089D800019B8CE7012806D15046FDF76BFE00226B
:1089E800164B1A6094E7164800F036FF90E74FF4EC
:1089F80080411048F8F7F4FE0028A5D0AAE700BF88
:108A08000C00002050090020C40F00206C1000202A
:108A18006D100020D40300203E0400206E100020BA
:108A2800D903002075BC0008B4BC00087BBC000852
:108A3800CC030020000402403D040020D0030020A5
:108A4800A8BC000800080240704710B5FF23044680
:108A5800221AD2B2914201D8184610BD14F8012B3F
:108A68005340082213F0800F02F1FF324FEA43030C
:108A780018BF83F0310312F0FF02DBB2F2D1E7E74F
:108A880030B5FF2305462C1AE4B2A14203D89B1A3D
:108A98005842584130BD15F8014B6340082413F083
:108AA800800F04F1FF344FEA430318BF83F031030A
:108AB80014F0FF04DBB2F2D1E5E70000002182B038
:108AC8000B4B00915A6C42F480425A645A6C02F47F
:108AD80080420092009A01911A6C42F080521A6406
:108AE8001B6C03F080530193019B02B0704700BFD9
:108AF800003802402DE9F043044689B014220021D1
:108B080003A800F0CCF92268224B9A423FD10025F5
:108B1800214C0095236B4FF0120943F004032363A3
:108B2800236B4FF0010803F004030093009B0195A9
:108B3800236B032743F001032363236B042603F00D
:108B480001030193019B4FF4007303A91348039396
:108B5800CDF81090CDF8148006970796F8F75EFDCB
:108B68004FF4807303A90E480393CDF81090CDF805
:108B7800148006970796F8F751FD0295236C43F485
:108B880000032364236C03F400030293029B09B0DF
:108B9800BDE8F083005C0040003802400008024055
:108BA800000002400268094B82B09A420BD10023B0
:108BB8000193074B1A6C42F010021A641B6C03F005
:108BC80010030193019B02B0704700BF00100040E2
:108BD8000038024070B5064688B01422002103A868
:108BE80000F05DF932682E4B9A4257D1002503F503
:108BF800F83301951A6C2B4842F480221A641A6CD7
:108C080003A902F480220192019A02951A6B264C5C
:108C180042F002021A631B6B03F002030293029BE9
:108C28004FF4406303930223049301230593032322
:108C3800069307230793F8F7F1FC4FF0006C1B4BE2
:108C4800204684E808104FF48063A560E56023613E
:108C58006561A561E56125626562F8F759FB08B1B0
:108C6800FFF7F2FE4FF060654FF0400E7463104B53
:108C7800A663104C4FF4806284E828400023204605
:108C8800E36022616361A361E36123626362F8F7D1
:108C98003FFB08B1FFF7D8FE3463A66308B070BD88
:108CA8000048004000040240640F00202860024091
:108CB800706002400C1000207047FEE7FEE7FEE7F8
:108CC800FEE7704770477047F8F77CBA0148F8F735
:108CD800EBBB00BF640F00200148F8F7E5BB00BFFD
:108CE8000C1000204FF48070F8F78CBD0148F9F79C
:108CF800EBBF00BFC80F002008B54FF48050F8F74D
:108D080081FD4FF40050F8F77DFD4FF48040F8F7EF
:108D180079FDBDE808404FF40040F8F773BD000046
:108D28000148F9F73FBC00BFD410002070B50E46CB
:108D380015460C46A31B9D4201DC284670BDAFF3C7
:108D4800008004F8010BF5E708B50A4B02461968DC
:108D580009B9094919606946186802448A4206D95E
:108D680000F068F80C2303604FF0FF3008BD1A606C
:108D780008BD00BF40040020341900204FF0FF3028
:108D880070474FF4005300204B6070470120704734
:108D98000020704700210C4B1A6842F001021A604B
:108DA80099601A6822F0847222F480321A60074AA5
:108DB8005A601A6822F480221A604FF00062D96063
:108DC800034B9A60704700BF0038024010300024FF
:108DD80000ED00E0002343600360836070470000FB
:108DE800DFF834D0002103E00C4B5B5843500431CA
:108DF8000B480C4B42189A42F6D30B4A02E0002368
:108E080042F8043B094B9A42F9D3FFF7C3FF00F03D
:108E180017F8FFF779FB704700000220A0BF000891
:108E280000000020DC010020DC01002034190020B3
:108E3800FEE70000014B1868704700BF0C000020D7
:108E480070B500250C4E0D4CA41BA410A54209D1E9
:108E580002F050FE00250A4E0A4CA41BA410A5429D
:108E680005D170BD56F8253098470135EEE756F81C
:108E7800253098470135F2E798BF000898BF0008E9
:108E880098BF00089CBF000810B5431E0A449142D1
:108E980000D110BD11F8014B03F8014FF7E7034665
:108EA8000244934200D1704703F8011BF9E7002BF5
:108EB8002DE9F0471E46BBBF03F100431E460023C1
:108EC8002D2388B0149F129927F02007462F1446A7
:108ED800109DDDF84CA00B7004D0452F00D1013552
:108EE800022300E0032307AA049206AA03928DE84E
:108EF80028042246334600F0E7FE472F804602D179
:108F0800119BDB0726D5462F08EB050911D198F8E8
:108F18000030302B0AD10022002320463146F7F7D3
:108F280077FD18B9C5F10105CAF80050DAF8003024
:108F380099440022002320463146F7F769FD38B9E5
:108F48003022079B994505D9591C07911A70F8E7F3
:108F5800CDF81C904046079B159AA3EB08031360B5
:108F680008B0BDE8F0870346F7B5002903F8022BDF
:108F7800B6BF2D222B2249420929427021DD0DF16D
:108F8800070217460A2691FBF6F506FB1511092D6F
:108F980001F1300102F8011C02F1FF34294609DC15
:108FA8003031023A04F8011CBA421C4604D3201A94
:108FB80003B0F0BD2246E6E712F8011B03F8011BD7
:108FC800F2E730221C46114404F8022B5970EEE7F0
:108FD8002DE9F04F91B00C461A9F93461E46054660
:108FE80001F0C2FD036818460993F7F7E9F8002372
:108FF8000E933B680A90073323F0070303F1080236
:1090080094F81880D4F800A03A60D3E90023C4E9A2
:109018001223D4F84C90A76C29F000430B934FF01F
:10902800FF32A64B38460B99F7F724FD002840F08D
:10903800F7814FF0FF32A14B38460B99F7F7FCFC4C
:10904800002840F0ED810022002338464946F7F712
:10905800E9FC10B12D2384F84330994B994FB8F1AE
:10906800470F98BF1F4603234FF0000923612AF0DA
:109078000403236000965B460FAA2146284600F0A9
:10908800DFF9013040F09A804FF0FF3011B0BDE8B1
:10909800F08F62680EA8531C0DF1340E4AF48063F9
:1090A80041D10622626000212360019363680DF1BB
:1090B80033020590029200933A464B460691CDF84A
:1090C8001080CDF80CE02846FFF7F1FE08F0DF032A
:1090D800472B074609D10D9BD81C02DB62689342D7
:1090E80059DDA8F102085FFA88F8B8F1650F0D9903
:1090F80036D80139424604F150000D91FFF733FF8D
:109108000E9A81468318012A236102DC2268D1075E
:1091180001D5013323619DF83330002BAAD02D23CC
:1091280084F84330A6E7B8F1670F02D0B8F1470FCB
:10913800B9D19AB1002106910DF133018DE80C00E7
:10914800236005903A46CDF81080CDF80CE00291E6
:109158004B462846FFF7ABFE0746BCE70122A1E7CE
:10916800B8F1660F19D1002963680CDD216113B9C4
:109178002268D20702D501330B4423610D9B4FF0BF
:109188000009A365C7E713B92268D00701D50233E0
:10919800F3E70123F1E74FF067080D9B0E9A93421E
:1091A80005DB22682361D107E8D50133E5E7002B09
:1091B800CCBF0123C3F102031344DEE723685A0539
:1091C80007D423693A4659462846B04701302AD180
:1091D8005AE7B8F1650F40F2DC80D4E912010022A9
:1091E8000023F7F715FC002839D00123364A5946E1
:1091F8002846B04701303FF447AF0E9B0D9A9A427C
:1092080002DB2368D8070ED50A9B099A59462846D7
:10921800B04701303FF438AF002704F11A080E9B1D
:10922800013B9F4211DB23689F0708D5002704F103
:109238001908E3680F9A9B1A9F42C0F2E780E0681A
:109248000F9B9842B8BF184620E70123424659466B
:109258002846B04701303FF417AF0137DFE70D9BD1
:10926800002B33DC0123184A59462846B047013001
:109278003FF40AAF0D9B23B90E9B13B92368D90796
:10928800D1D50A9B099A59462846B04701303FF480
:10929800FBAE4FF0000804F11A090D9B5B4298459C
:1092A80001DB0E9B8EE701234A4659462846B04704
:1092B80001303FF4E9AE08F10108EEE7FFFFEF7F68
:1092C800D4BC0008D8BC0008E4BC00080E9AA36D02
:1092D8009A42A8BF1A46002A904636DC4FF0000A88
:1092E80004F11A0328EAE8780B93D4F85890A9EB0C
:1092F80008039A4531DB0E9B0D9A9A4238DB2368A6
:10930800DA0735D40E9B0D99A3EB0902A3EB0108EC
:109318009045A8BF9046B8F1000F31DC002728EA35
:10932800E87804F11A090D9A0E9B9B1AA3EB08031F
:109338009F42BFF678AF01234A4659462846B047B0
:1093480001303FF4A1AE0137EDE7134659463A46DE
:109358002846B0470130C1D196E601230B9A5946F9
:109368002846B04701303FF48FAE0AF1010ABCE746
:109378000A9B099A59462846B0470130C2D183E66C
:10938800434607EB090259462846B0470130C5D184
:109398007AE60E9A012A01DCDB0734D501233A4626
:1093A80059462846B04701303FF46EAE0A9B099AE9
:1093B80059462846B04701303FF466AED4E9120159
:1093C80000220023F7F724FB50B1002704F11A0804
:1093D8000E9B013B9F420CDB4B4604F15002F2E628
:1093E8000E9B7A1C013B59462846B0470130F3D101
:1093F8004AE60123424659462846B04701303FF421
:1094080043AE0137E4E701233A46ECE7012342463D
:1094180059462846B04701303FF436AE013708E7D1
:109428003A464B4638464946F7F724FB00283FF4AE
:1094380030AE014B014F12E6DCBC0008E0BC00086E
:109448002DE9F04791461F468A680B690646934204
:10945800B8BF1346C9F8003091F843200C46DDF830
:10946800208012B10133C9F800302368990642BF41
:10947800D9F800300233C9F80030256815F0060520
:1094880007D104F1190AE368D9F800209B1A9D4214
:109498002ADB94F843302268003318BF0123920670
:1094A8002FD404F1430239463046C047013022D058
:1094B8002368E56803F00603042B18BF0025D9F8D4
:1094C80000204FF0000908BFAD1AA368226908BF41
:1094D80025EAE5759342C4BF9B1AED181A344D4529
:1094E8001BD10020BDE8F08701235246394630469B
:1094F800C047013003D14FF0FF30BDE8F087013598
:10950800C1E73020E11881F843005A1C94F845104F
:109518002244023382F84310C3E701232246394626
:109528003046C0470130E6D009F10109D7E700000D
:109538002DE9F04317460A7E85B06E2A98460646FE
:109548000C460C9B01F1430E00F0BC801AD8632A2C
:109558002ED00AD8002A00F0C880582A00F08A8045
:1095680004F1420584F842202AE0642A01D0692ADD
:10957800F6D121681A6811F0800F23D0111D1960E7
:10958800136827E0732A00F0B48008D86F2A2AD01D
:10959800702AE5D10A6842F020020A6003E0752AC1
:1095A80021D0782ADCD178226F4984F8452064E0FC
:1095B8001A6801F14205111D1960136884F84230D8
:1095C8000123A3E011F0400F02F104011960D7D084
:1095D800B2F90030002B03DA2D225B4284F84320D5
:1095E80062490A2217E02068196810F0800F03D03A
:1095F800081D18600B6806E010F0400F01F1040028
:109608001860F7D00B886F2A14BF0A22082257491E
:10961800002084F843006568002DA560C0F29C8096
:10962800206820F004002060002B3FD1002D40F07E
:1096380095807546082A0BD12368DA0708D523696F
:1096480062689A42DEBF302305F8013C05F1FF3518
:10965800AEEB05032361CDF800803B4603AA214603
:109668003046FFF7EDFE013055D14FF0FF3005B021
:10967800BDE8F08381F845203C492268186812F05B
:10968800800F00F104051D6001D0036802E0550653
:10969800FBD50388D00744BF42F0200222601BB9E3
:1096A800226822F0200222601022B1E77546B3FB3F
:1096B800F2F002FB1033CB5C05F8013D03460028AD
:1096C800F5D1B7E708681A6810F0800F496904D027
:1096D800101D18601368196007E010F0400F02F1C0
:1096E800040018601368F6D01980002375462361BA
:1096F800B1E71A68111D19601568002162682846CB
:1097080001F0ACFA08B1401B606063682361002374
:1097180084F843309FE723692A4639463046C047D4
:109728000130A2D023689B0707D5002504F1190949
:10973800E368039A9B1A9D4205DBE068039B984205
:10974800B8BF184693E701234A4639463046C04712
:1097580001308AD00135EBE7002BA7D10B7804F153
:10976800420584F8423065E7F7BC0008E6BC00080B
:109778000FB40A4B13B51C6824B1A36913B920466A
:1097880001F068F905AB049AA1682046019301F03D
:1097980075FF02B0BDE8104004B070470C0000200F
:1097A80070B50E46054618B183690BB901F052F938
:1097B800AB69AC6813B9284601F04CF9234B9C42BD
:1097C80017D16C68A3891B071DD52369DBB1013E3E
:1097D800A36816F8011F013BA360E9B9002B2EDA34
:1097E80022460A21284600F021F9013011D00A202A
:1097F80070BD174B9C4201D1AC68E3E7154B9C4206
:1098080008BFEC68DEE72146284600F061F9002829
:10981800DDD04FF0FF3070BD002B04DAA26993420F
:1098280006DB0A2904D023685A1C22601970CFE786
:109838002246284600F0FAF80130C9D1E9E70A20A3
:1098480023685A1C2260187070BD00BF38BD00081C
:1098580058BD000818BD0008024B01461868FFF7FC
:109868009FBF00BF0C00002000294FF480630CBF8D
:109878000222002200F000B82DE9F7431D46514BA3
:1098880004461E680F46904626B1B36913B93046A0
:1098980001F0E0F84C4B9C4252D17468B8F1020FC9
:1098A80006D0B8F1010F00F28980002DC0F2868041
:1098B8002146304601F064F8616B41B104F144037C
:1098C800994202D0304601F0B7FC002363630023BD
:1098D800A3616360A3891B0603D52169304601F0A3
:1098E800ABFCA389B8F1020F23F44A6323F0030306
:1098F800A3815DD001AB6A462146304601F042F9AA
:10990800A3891843A0812DBB009D284601F09EF92C
:10991800074600284ED1DDF80090A9453CD14FF00C
:10992800FF30A38943F00203A3810023A36004F15D
:109938004703236023610123636103B0BDE8F0831B
:10994800224B9C4201D1B468A8E7214B9C4208BF36
:10995800F468A3E7002FD8D0B36913B9304601F0F3
:1099680079F8B8F1010F08BFA389276004BF43F055
:109978000103A381A389276113F0080065611BD047
:1099880013F001004FF000031FBF6D42A360A561F3
:10999800184608BFA560D0E7484601F057F90746C2
:1099A8000028BCD0A3894D4643F08003A381D3E7A8
:1099B8000020B6E7A946F5E7A060BEE74FF0FF3004
:1099C800BBE700BF0C00002038BD000858BD0008E8
:1099D80018BD00080EB44FF4027100B59CB0ADF884
:1099E80014106FF00041049107914FF6FF711DAB01
:1099F80002900690084853F8042BADF8161000683A
:109A080002A9019301F01EFD0022029B1A701CB0EE
:109A18005DF804EB03B070470C000020034611F812
:109A2800012B03F8012B002AF9D17047F8B50E462F
:109A38001446054618B183690BB901F00BF8214BA0
:109A48009C422AD16C68A369A360A3891A072ED502
:109A5800236963B323692068F6B2C01A636937467D
:109A6800984204DB2146284600F08AFF28BBA368F9
:109A78000130013BA36023685A1C22601E70636991
:109A8800984204D0A389DB0719D50A2E17D121469D
:109A9800284600F075FF90B10FE00B4B9C4201D1B6
:109AA800AC68D0E7094B9C4208BFEC68CBE721467D
:109AB800284600F00DF80028CCD04FF0FF37384684
:109AC800F8BD00BF38BD000858BD000818BD000823
:109AD800324B70B51D6806460C4625B1AB6913B903
:109AE800284600F0B7FF2E4B9C420FD16C68B4F9A2
:109AF8000C309AB215072CD4D00611D40922326042
:109B080043F04003A3814FF0FF3070BD254B9C42CA
:109B180001D1AC68EBE7244B9C4208BFEC68E6E750
:109B2800510712D5616B41B104F14403994202D047
:109B3800304601F081FB00236363A38923F02403EB
:109B4800A3810023636023692360A38943F008038A
:109B5800A38123694BB9A38903F42073B3F5007F6C
:109B680003D02146304601F031F8A28912F00103F2
:109B78000CD00023A36063695B42A361236953B9D6
:109B8800B4F90C3013F08000BAD170BD920758BFF9
:109B98006369A360F2E70020F7E700BF0C0000202C
:109BA80038BD000858BD000818BD00082DE9F74F5A
:109BB80003690C6980469C4200F38280013C01F1F4
:109BC800140700F1140657F8245056F824000135FC
:109BD800B0FBF5F54FEA840E06EB0E0307EB0E0912
:109BE80001938DB34FF0000A3846B446D34650F877
:109BF800042B93B205FB03A3120C4FEA134A05FB8F
:109C080002A29BB2ABEB0303BCF800B04FEA124AC6
:109C18005B441FFA82FBDCF800208145CBEB124243
:109C280002EB23429BB243EA02434FEA224B4CF831
:109C3800043BDCD256F80E3033B9019B043B9E42FC
:109C48001A4631D3C8F81040404601F01EFA0028E1
:109C580026DB30464FF0000E013557F8041BD0F8CC
:109C680000C08BB2AEEB03031FFA8CF213440A0C4C
:109C7800C2EB1C4202EB23429BB243EA0243B945C2
:109C88004FEA224E40F8043BE7D256F8242006EB70
:109C980084032AB9043B9E421A460BD3C8F81040E5
:109CA800284603B0BDE8F08F1268043B002AC9D1EA
:109CB800013CC4E71268043B002AEFD1013CEAE703
:109CC8000020EEE7000000002DE9F04F466A95B04D
:109CD8000446219DCDE902233EB9102000F0B6FFCD
:109CE8006062466086600660C660636A196851B142
:109CF8005A68012393404A608B60204600F0F0FFC9
:109D08000022636A1A60039B002BB7BF012300235C
:109D18002B60039BAEBF2B6023F000430393DDF859
:109D28000C90AB4B33EA09031BD142F20F73209A14
:109D38001360029B23B9C9F31300002800F0838540
:109D4800229B53B9A34B21E0A34B06930833229AD5
:109D58001360069815B0BDE8F08F9E4B0693033349
:109D6800F5E7DDE902670022002330463946F6F7B9
:109D78004FFE804660B10123209A1360229B002B7E
:109D880000F05E85954B229A1360013B0693E0E74D
:109D980012AB019313AB009332463B46204601F0C9
:109DA800EDF9C9F30A558246002D7DD03046C7F338
:109DB800130343F07F5141F44011A5F2FF35CDF86C
:109DC80040800022864BF6F707FA7BA3D3E90023ED
:109DD800F6F7B6FB7AA3D3E90023F6F7FFF90646B0
:109DE80028460F46F6F746FB77A3D3E90023F6F794
:109DF800A7FB02460B4630463946F6F7EFF906460A
:109E08000F46F6F74DFE00228346002330463946BA
:109E1800F6F708FE58B15846F6F72CFB02460B46F3
:109E280030463946F6F7F4FD08B90BF1FF3BBBF1B4
:109E3800160F58D8DDE902236A4901EBCB01D1E9B5
:109E48000001F6F70DFE00284FD000230BF1FF3B71
:109E58000D93129B5D1B6B1E079343BF0023C5F137
:109E6800010807934FF00008BBF1000F3FDB079B89
:109E7800CDF830B05B440793002308931E9B092B51
:109E880000F2B480052BC4BF043B1E931E9BC8BFC1
:109E98000026A3F10203D8BF0126032B00F2B280EB
:109EA800DFE803F084862D78139B129D1D4405F28C
:109EB8003243202B11DD029A05F21240C3F1400310
:109EC80022FA00F009FA03F31843F6F7C3FA01235C
:109ED800A1F1F871013D109373E7C3F12000029BD3
:109EE80003FA00F0F1E70123B2E70D90B1E7CBF1F7
:109EF800000308930023A8EB0B080C93BEE701238B
:109F080009931F9B002B40F38080994604930022FD
:109F18000421656A6A6001F114029A427AD9696873
:109F2800204600F0A9FE636A28601B68B9F10E0F8D
:109F3800069300F2F080002E00F0ED80DDE90223A8
:109F4800BBF1000FCDE90E2379DD264A0BF00F0394
:109F58004FEA2B1602EBC303F006D3E90023CDE941
:109F68000A235CD5DDE90E011F4B0325D3E908233D
:109F7800F6F710FCCDE9020106F00F061A4F002E85
:109F88004FD1DDE90A23DDE90201F6F703FCCDE94B
:109F980002016EE0012309931F9B5B4403F1010951
:109FA80004934B46012BB8BF0123B0E70023A7E772
:109FB8000023F0E7AFF3008061436F63A787D23FC8
:109FC800B3C8608B288AC63FFB799F501344D33FA0
:109FD8000000F07F11BD000808BD0008E5BC0008BE
:109FE8000000F83FA0BD000878BD00080126002346
:109FF80009961E934FF0FF330022049399461223CB
:10A008001F9284E701230993F4E7012304939946F7
:10A018001A46F5E76A68490001326A607BE702255B
:10A02800ACE7F10708D5DDE90A01D7E90023F6F71F
:10A0380087FACDE90A010135761008379FE700F065
:10A04800A580DDE90E01CBF10006A24B06F00F0258
:10A0580003EBC203D3E90023F6F772FA02250023C3
:10A06800CDE902019C4F3611002E40F08480002B70
:10A078008DD10D9B002B00F08B80DDE90223CDE90B
:10A088000A23DDE90A010022944BF6F7CBFC0028ED
:10A098007ED0B9F1000F7BD0049B002B37DDDDE9C2
:10A0A8000A0100228E4BF6F74BFACDE90201049E15
:10A0B8000BF1FF3701352846F6F7DCF9DDE9022315
:10A0C800F6F73EFA874B0022F6F788F8CDE90A0141
:10A0D8000B9BA3F150750B95002E5CD1DDE90201B5
:10A0E8000022814BF6F778F80A9A2B46CDE902014F
:10A0F800F6F7B6FC002840F0F782DDE902010A9A7B
:10A1080005F10043F6F78EFC002840F0EB82DDE90C
:10A118000E23CDE90223139B002BC0F25081BBF123
:10A128000E0F00F34C816B4B03EBCB03D3E90023F9
:10A13800CDE904231F9B002B80F2DA80B9F1000FD0
:10A1480000F3D68040F0CD82DDE904010022664BA1
:10A15800F6F7F6F9DDE90223F6F778FC4E464F46A6
:10A16800002840F0A482069B069A5D1C31230BF15F
:10A17800010B13709FE2F20705D5D7E90023F6F724
:10A18800DFF901230135761008376DE7022570E7FE
:10A198005F464E468FE7069A4E4B32441192099A13
:10A1A800711E002A48D003EBC103D3E90023002025
:10A1B8004E49F6F7EFFADDE90A23F6F70DF8CDE98F
:10A1C8000A01069DDDE90201F6F76AFC0646F6F784
:10A1D80051F902460B46DDE90201F5F7FDFFDDE91D
:10A1E8000A23303605F8016BCDE90201F6F71AFCAF
:10A1F800002864D1DDE9022300203849F5F7ECFF97
:10A20800DDE90A23F6F70EFC002840F0B980119B1F
:10A218009D423FF47CAFDDE90A010022304BF6F79E
:10A228008FF90022CDE90A01DDE902012C4BF6F78E
:10A2380087F9CDE90201C5E703EBC101D1E90001C6
:10A24800DDE90A23F6F77CF9CDE90A01069DDDE987
:10A258000201F6F725FC0646F6F70CF902460B460E
:10A26800DDE90201F5F7B8FF3036119B05F8016BFF
:10A27800AB42CDE902014FF0000224D11B4BDDE9CE
:10A288000A01F5F7ABFF02460B46DDE90201F6F7D6
:10A29800E7FB002874D1DDE90A2300201349F5F70C
:10A2A8009BFF02460B46DDE90201F6F7BBFB0028DF
:10A2B8003FF42DAF15F8013C6A1E302B01D0BB4688
:10A2C8004DE01546F6E7064BF6F73AF9CDE90201F7
:10A2D800BDE700BFA0BD000878BD00080000F03F42
:10A2E8000000244000001C40000014400000E03F33
:10A2F800069DDDE90267DDE9042330463946F6F7B5
:10A3080049FAF6F7CDFB8046F6F7B4F8DDE9042301
:10A31800F6F716F902460B4630463946F5F75CFF64
:10A3280008F1300605F8016B069E0246AE1BB145E2
:10A338000B4637D1F5F752FF06460F4602460B4645
:10A34800DDE90401F6F76EFBC8B9DDE90401324620
:10A358003B46F6F75DFB10B118F0010F0FD15146DF
:10A36800204600F0BDFC0023209A2B700BF101035E
:10A378001360229B002B3FF4ECAC1D60E9E45F46C0
:10A3880015F8012C6B1E392A06D1069A9A4207D174
:10A3980030231370134601371A7801321A708EE78A
:10A3A8001D46EDE70022B54BF6F7CAF80022002358
:10A3B80006460F46F6F72CFB00289CD0CFE7099AF3
:10A3C800002A00F029811E9A012A00F30E81109AB2
:10A3D800002A00F0068103F233434546089E079A97
:10A3E80001211A4420469844079200F019FD0746B7
:10A3F800002D0BDD079B002B08DDAB42A8BF2B46C9
:10A40800079AA8EB0308ED1AD31A0793089BFBB128
:10A41800099B002B00F00481002E11DD39463246DD
:10A42800204600F093FD524601460746204600F0BC
:10A4380000FD51460A90204600F052FC0A9B9A46BD
:10A44800089B9A1B04D05146204600F07FFD8246A7
:10A458000121204600F0E4FC0C9B0646002B40F34B
:10A46800E1801A460146204600F070FD1E9B064614
:10A47800012B40F3DA8000230893336906EB83034A
:10A48800186900F07FFCC0F12000079B184410F009
:10A498001F0000F0F080C0F12003042B40F3E2809D
:10A4A800079BC0F11C008044054403440793B8F19E
:10A4B800000F05DD51464246204600F095FD8246D4
:10A4C800079B002B05DD31461A46204600F08CFD1F
:10A4D80006460D9B002B00F0D3803146504600F015
:10A4E800D4FD002880F2CC80002351460A22204661
:10A4F80000F00DFC099B0BF1FF3B8246002B00F09E
:10A50800A981002339460A22204600F000FC049B5A
:10A518000746002B03DC1E9B022B00F3B980002D9D
:10A5280005DD39462A46204600F05EFD0746089BB1
:10A53800002B00F010817968204600F09DFB05464D
:10A548003A6907F10C01023292000C30FEF79CFCCC
:10A5580001222946204600F047FD07970746029B3F
:10A56800DDF8188003F00103089331465046FFF7E1
:10A578001DFB0799054600F13009504600F085FD9E
:10A588003A4602903146204600F099FDC3680246DB
:10A59800002B40F0E28001460990504600F075FD1E
:10A5A8000346099A11462046099300F099FB099B36
:10A5B800002B40F0D4801E9A002A40F0D080089AE0
:10A5C800002A40F0CC80B9F1390F00F0E880029BF6
:10A5D800002B01DD05F1310908F1010588F800902B
:10A5E8006BE0129BC3F13603F7E6089B09F1FF36CF
:10A5F800B342B7BF089B9E1BF21A0C9BBFBF0896BD
:10A608009B180C930026B9F1000FB9BFA8EB0905F8
:10A61800002345464B46E2E6089E4546099FE7E685
:10A62800089A10E71E9B012B18DC029BB3B9039B09
:10A63800C3F31303A3B9039B23F000431B0D1B05AE
:10A648002BB1079B08F101080133079301230893F5
:10A658000C9B002B7FF411AF012016E70023F6E7CF
:10A66800029BF4E73FF423AF079A1C331A4498443B
:10A678001D4413461AE70346F6E700BF00002440CE
:10A68800B9F1000F33DC1E9B022B30DDCDF81090A2
:10A69800049B63B931460522204600F038FB014689
:10A6A8000646504600F0F1FC00283FF75CAD1F9BC2
:10A6B800069D6FEA030B002307933146204600F0FE
:10A6C8000FFB002F3FF44BAE079B2BB1BB4203D0CF
:10A6D8001946204600F004FB3946204600F000FBEE
:10A6E8003DE600263746E2E7BB4637463BE5099B91
:10A6F800CDF81090002B7FF412AF069D31465046DE
:10A70800FFF754FA069B00F1300905F8019B049AFB
:10A71800EB1A9A4200F38180069B012AACBF9B1872
:10A72800013398460023079351460122204600F042
:10A738005BFC3146824600F0A8FC002834DC02D1DC
:10A7480019F0010F30D1454615F8013C6A1E302B2F
:10A75800B3D11546F8E73846FFE6012322E7029A07
:10A76800002A04DB28D11E9A32BB089A22BB002B90
:10A778007FF732AF51460122204600F035FC3146C2
:10A78800824600F082FC002805DC7FF425AF19F032
:10A79800010F3FF421AFB9F1390F7FF41BAF392313
:10A7A80008F1010808F8013C454615F8013C6A1E05
:10A7B800392B3AD001333FE0002B08F1010505DDC4
:10A7C800B9F1390FEBD009F1010907E7069B049AA3
:10A7D800EB1A9342A84605F8019CA5D051460023E0
:10A7E8000A22204600F093FA079B8246BB424FF0AC
:10A7F8000A024FF000030799204604D100F087FAB7
:10A8080007900746B1E600F082FA002307900A2273
:10A818003946204600F07BFAF3E7514600230A2226
:10A82800204600F074FA824668E7069B934205D1F9
:10A838003123069A0BF1010B13703EE71546B4E776
:10A84800094BFFF7A3BA229B002B7FF47DAA074B85
:10A85800FFF79CBA049B002B3FF74FAF1E9B022BC0
:10A868007FF74BAF14E700BFE4BC000808BD000841
:10A878008A892DE9F041054610070C465AD44B68E1
:10A88800002B05DC0B6C002B02DC0020BDE8F081FE
:10A89800E66A002EF9D0002312F480522F682B604C
:10A8A80033D0606DA3895A0705D56368C01A636BF6
:10A8B8000BB1236CC01A00230246E66A216A2846B7
:10A8C800B047431CA38906D129681D294BD82B4AB8
:10A8D800CA40D60747D5002262602269D90422609F
:10A8E80004D5421C01D12B6803B96065616B2F60E8
:10A8F8000029CAD004F14403994202D0284600F046
:10A908009BFC00206063BDE8F081216A0123284692
:10A91800B047411CC6D12B68002BC3D01D2B01D0DA
:10A92800162B01D12F60B0E7A38943F04003A38120
:10A93800BDE8F0810F69002FA7D0930718BF002347
:10A948000E6808BF4B69A6EB07080F608B60B8F16B
:10A95800000F9ADD43463A46216A2846A66AB04760
:10A96800002807DCA38943F04003A3814FF0FF30A0
:10A97800BDE8F0810744A8EB0008E8E701004020A3
:10A9880038B50B6905460C46DBB118B183690BB9BC
:10A9980000F060F80C4B9C4209D16C68B4F90C309B
:10A9A8007BB121462846BDE83840FFF761BF074B19
:10A9B8009C4201D1AC68F1E7054B9C4208BFEC68AA
:10A9C800ECE7002038BD00BF38BD000858BD0008BE
:10A9D80018BD0008014900F0A9B800BF89A90008FE
:10A9E800002310B504460360436083608181436699
:10A9F800C281036143618361194608225C30FEF716
:10AA08004EFA054B24626362044BA362044BE36273
:10AA1800044B236310BD00BFD1B80008F3B8000889
:10AA28002BB900084FB9000870B568254A1E554370
:10AA38000E4605F1740100F04BFC044640B10021BC
:10AA480080E842000C30A06005F16802FEF727FAA2
:10AA5800204670BD836910B5044633BB8364C36464
:10AA68000365124B124A1B688262984204BF012395
:10AA7800836100F01FF86060204600F01BF8A060BA
:10AA8800204600F017F80022E06004216068FFF714
:10AA9800A7FF01220921A068FFF7A2FF02221221C5
:10AAA800E068FFF79DFF0123A36110BDD0BC00083B
:10AAB800DDA90008F8B51C4B07461E68B36913B931
:10AAC8003046FFF7C7FF4836B4687368013B03D5C3
:10AAD800336833B13668F7E7B4F90C506DB16834B0
:10AAE800F4E704213846FFF79FFF30600028F1D1D2
:10AAF8000C2304463B602046F8BD4FF6FF73E38104
:10AB080001236566A3812560A5606560256165618F
:10AB1800A5610822294604F15C00FEF7C0F96563C7
:10AB2800A563A564E564E6E7D0BC00082DE9F84311
:10AB380080468946002600F1480414B93046BDE82D
:10AB4800F883A5686768013F01D52468F5E7AB89F4
:10AB5800012B07D9B5F90E30013303D029464046F9
:10AB6800C84706436835EEE7044B1B68186A044B70
:10AB7800002808BF1846F030704700BF0C000020BE
:10AB88007000002070B50E46B1F90E1090B0002983
:10AB980014461D4607DA00232B60B3891A0610D421
:10ABA8004FF480630EE001AA00F0F4FE0028F2DB07
:10ABB800029A02F47042A2F500535A425A412A609E
:10ABC800EEE740230020236010B070BD8B8973B579
:10ABD8009D0706460C4607D504F147032360236109
:10ABE8000123636102B070BD01AB6A46FFF7CAFF7B
:10ABF80000990546304600F06BFB48B9B4F90C30B3
:10AC08009A05EFD423F0030343F00203A381E3E79B
:10AC18000D4BB362A389206043F08003A381009B9E
:10AC280020616361019B5BB1B4F90E10304600F0FE
:10AC3800C3FE28B1A38923F0030343F00103A381D2
:10AC4800A3891D43A581CDE7DDA90008024B014674
:10AC5800186800F03DBB00BF0C00002010B5C9B259
:10AC680002449042034601D1002010BD1C780130F7
:10AC78008C42F6D1184610BD70B5456A04460E469A
:10AC88003DB91020FFF7E2FF60624560856005600E
:10AC9800C560656AEB6883B1636ADB6853F82600B0
:10ACA800B8B9012101FA06F56A1D9200204600F0A4
:10ACB800B4FA60B1466085600EE021220421204686
:10ACC80000F0ABFA636AE860DB68002BE4D100208F
:10ACD80070BD026843F8262000230361C36070BD7D
:10ACE80070B5446A06460D463CB91020FFF7AEFF22
:10ACF8007062446084600460C4603DB1736A6A68CD
:10AD0800DB6853F82210296043F8225070BD2DE902
:10AD1800F0411F4606460C4600230D6901F1140E4A
:10AD2800DEF80000013381B202FB0171000C0F0C48
:10AD380002FB007089B201EB00419D424FEA1047C7
:10AD48004EF8041BECDCD7B1A3689D4212DB6168A6
:10AD580030460131FFF790FF8046226904F10C016B
:10AD6800023292000C30FEF78FF821463046FFF78A
:10AD7800B7FF444604EB850301355F612561204632
:10AD8800BDE8F081020C12040346B2B90304102096
:10AD980013F07F4F04BF1B02083013F0704F04BF3D
:10ADA8001B01043013F0404F04BF9B000230002BFE
:10ADB80006DB5B0003D5013070470020E8E7202060
:10ADC80070470368014613F007020BD0DA0723D453
:10ADD800980749BF5B089B0801200B605CBF0B60AC
:10ADE8000220704798B2A8B910201B0C13F0FF0F6F
:10ADF80004BF1B0A08301A0704BF1B0904309A074E
:10AE080004BF9B080230DA0702D45B0806D0013081
:10AE18000B6070471046E9E7002070472020704714
:10AE280010B50C460121FFF727FF0122446102619A
:10AE380010BD2DE9F74F14460A69236989469A42DD
:10AE4800BEBF0B46A1461C46D9F81070D4F810A016
:10AE5800D9F80830D9F8041007EB0A069E42C8BF93
:10AE68000131FFF709FF00F114052B46002205EB1D
:10AE78008608434516D304F1140209F1140102EBC4
:10AE88008A0301EB87070193019C134694420CD86F
:10AE9800002E03DD58F8043D002B54D0066103B0A2
:10AEA800BDE8F08F43F8042BE3E7B3F800A00432C1
:10AEB800BAF1000F20D0AE4689464FF0000C59F881
:10AEC800044BBEF800B0A3B20AFB03B34FEA144B1D
:10AED800DEF8004063444FEA144C0AFB0BC404EB51
:10AEE80013449BB243EA04434F454FEA144C4EF8CF
:10AEF800043BE4D8CEF800C032F8029CB9F1000F48
:10AF08001FD0AE468C464FF0000A2B68BCF80040B4
:10AF1800BEF802B09BB209FB04B4A24443EA0A4358
:10AF28004EF8043B5CF8043BBEF800401B0C09FBE0
:10AF38000343674503EB1A434FEA134AE6D8CEF8B2
:10AF480000300435A0E7013EA2E700002DE9F843F0
:10AF5800154612F0030206460F4607D0214C013A67
:10AF6800002354F82220FFF7D2FE0746AD1035D053
:10AF7800746A3CB91020FFF769FE7062446084600F
:10AF88000460C460D6F82480D8F808404CB940F270
:10AF980071213046FFF744FF00230446C8F8080033
:10AFA80003604FF00008EB070AD5394622463046C1
:10AFB800FFF73FFF814639463046FFF791FE4F467F
:10AFC8006D100BD0206838B9224621463046FFF76D
:10AFD80030FF2060C0F800800446E4E73846BDE84A
:10AFE800F88300BF68BE00082DE9F0470C46074605
:10AFF800164623694FEA621A0AEB03094968A368EF
:10B0080009F10105AB4231DB3846FFF735FE002276
:10B018008046114600F1140352452ADB20692AEACA
:10B02800EA7A04F1140116F01F0203EB8A0301EB1C
:10B03800800E22D00020C2F1200C0E6896403043CA
:10B0480043F8040B51F8040B8E4520FA0CF0F4D8A1
:10B05800186008B109F10205013D3846C8F81050DA
:10B068002146FFF73DFE4046BDE8F08701315B0011
:10B07800C8E743F822100132CEE7043B51F8042B0D
:10B088008E4543F8042FF9D8E6E703690A6930B515
:10B098009B1A0CD19200143014318418114454F8BE
:10B0A800045D51F8042D954203D005D301231846B9
:10B0B80030BDA042F3D3FAE74FF0FF33F7E72DE9AD
:10B0C800F0470D460746114628461446FFF7DDFFB0
:10B0D800061E08D131463846FFF7CEFD01234661EA
:10B0E8000361BDE8F087A4BF23462C463846616853
:10B0F800A6BF1D4600260126FFF7BEFD4FF0000C37
:10B10800C6602B69266904F1140205F1140902EBE3
:10B11800860709EB830800F1140152F804AB59F8CB
:10B12800045B1FFA8AF36344ACB21B1B2C0CC4EB00
:10B138001A4404EB23449BB24FEA244CC84543EA23
:10B148000444964641F8044BE7D8BE4505D351F868
:10B15800043D8BB10661BDE8F0875EF8044BA2B2EE
:10B168006244131403EB144392B242EA03424FEAD7
:10B17800234C41F8042BE8E7013EE8E72DE9F341C9
:10B188001C4601219046089E099DFFF775FDC4F3F2
:10B198001302C4F30A54074634BB0192B8F1000FF6
:10B1A80027D002A840F8088DFFF70BFE0099F0B1F0
:10B1B800019AC0F1200302FA03F30B43C2407B61FA
:10B1C8000192019B002B14BF02210121BB6139614F
:10B1D800C4B1A4F2334404443460C0F1350028609B
:10B1E800384602B0BDE8F08142F48012D5E77961B3
:10B1F800E7E701A8FFF7E5FD0121019B39617B61C4
:10B208002030E5E7A0F2324007EB8103306018698F
:10B21800FFF7B8FDC0EB4110E1E738B502FB01F4D8
:10B22800214600F055F8054618B122460021FDF7E1
:10B2380036FE284638BD000038B50546002943D0FB
:10B2480051F8043C0C1F002BB8BFE41800F002FCB6
:10B258001E4A1368104633B9636014602846BDE877
:10B26800384000F0F8BBA3420BD92168621893421A
:10B2780001BF1A685B685218226063600460EDE7DA
:10B2880013465A680AB1A242FAD919685818A04256
:10B298000BD120680144581882421960DED1106829
:10B2A8005268014419605A60D8E702D90C232B6010
:10B2B800D4E7206821188A4201BF1168526809182A
:10B2C800216062605C60C9E738BD00BF44040020AB
:10B2D80070B5CD1C25F0030508350C2D38BF0C259D
:10B2E800002D064601DBA94203D90C233360002058
:10B2F80070BD00F0AFFB234A1468214691B9224C77
:10B3080023681BB9304600F0CFFA20602946304642
:10B3180000F0CAFA431C26D10C233046336000F0F3
:10B328009AFBE4E70B685B1B1AD40B2B0FD90B6055
:10B33800CC18CD50304600F08EFB04F10B00231DD5
:10B3480020F00700C31A1BD05A42E25070BD8C424D
:10B358000BBF63684B681360636018BF0C46E9E76E
:10B368000C464968CAE7C41C24F00304A04205D06F
:10B37800211A304600F098FA0130CDD02560D9E77F
:10B3880070BD00BF44040020480400202DE9F047A8
:10B398008E6882469E420C469146984635D88A89E0
:10B3A80012F4906F31D00223256809696F1A656914
:10B3B80005EB450595FBF3F508F101033B449D4278
:10B3C80038BF1D46530531D52946FFF781FF06468C
:10B3D80050B90C23CAF80030A3894FF0FF3043F06E
:10B3E8004003A381BDE8F0873A462169FDF74CFD8B
:10B3F800A38923F4906343F08003A38126613E442C
:10B40800266046466561ED1BA560464528BF464651
:10B4180049463246206800F003FBA36800209B1BC6
:10B42800A36023681E442660BDE8F0872A4600F022
:10B4380013FB06460028E1D121695046FFF7FCFEC0
:10B44800C7E700002DE9F04F9DB003938B89804634
:10B458001C060D4616460FD50B696BB94021FFF740
:10B4680037FF2860286128B90C23C8F800304FF04E
:10B47800FF30C4E040236B610023099320238DF83B
:10B48800293030234FF0010B8DF82A3037463C46DF
:10B4980014F8013B002B3CD1B7EB060A0BD05346FE
:10B4A800324629464046FFF771FF013000F0A2807E
:10B4B800099B534409933B78002B00F09B800023A1
:10B4C8004FF0FF3204930793059206938DF853309B
:10B4D8001A93052221785048FFF7C0FB671C049B8C
:10B4E800D8B9D90644BF20228DF853201A0744BF83
:10B4F8002B228DF8532022782A2A16D000210A20E0
:10B50800079A27463B780134303B092B50D9C9B1FB
:10B5180011E0252BC0D02746B9E73F4A3C46801AA0
:10B528000BFA00F018430490D3E7039A111D126830
:10B538000391002A01DB079204E0524243F0020320
:10B54800079204933B782E2B0DD17B78791C2A2BFC
:10B5580032D1039B02371A1D1B680392002BB8BF18
:10B568004FF0FF3305932D4C032239782046FFF71F
:10B5780075FB38B14023001B03FA00F0049B013728
:10B58800034304933978062225487E1C8DF8281039
:10B59800FFF764FB002835D0224BFBB9039B073328
:10B5A80023F0070308330393099B4B4409936DE782
:10B5B80000FB02320121A4E700230A241846059360
:10B5C8000F463A780131303A092A03D9002BCAD0FC
:10B5D8000590C8E704FB00200123F1E703AB0093C3
:10B5E8002A46114B04A94046FDF7F2FCB0F1FF3F93
:10B5F8008146D9D1AB895B063FF539AF09981DB0B3
:10B60800BDE8F08F03AB00932A46074B04A94046D8
:10B61800FDF78EFFEAE700BF74BE00087ABE000897
:10B628007EBE0008D98F000895B30008936810B44F
:10B63800013B002B936008DA9469A34202DBCBB28A
:10B648000A2B02D110BCFEF7F1B91368581C106020
:10B658001970C8B210BC7047F8B506460F461446B4
:10B66800D518AC4201D1002007E03A4614F8011B76
:10B678003046FFF7DBFF431CF3D1F8BD2DE9F04F4F
:10B688009DB00C4617460393064618B183690BB95B
:10B69800FFF7E0F97C4B9C4257D17468A3891807DF
:10B6A8005DD52369002B5AD00023099320238DF8F8
:10B6B800293030234FF0010B8DF82A30B846454623
:10B6C80015F8013B002B55D1B8EB070A0BD05346B0
:10B6D8003A4621463046FFF7BFFF013000F0C480EC
:10B6E800099B5344099398F80030002B00F0BC8064
:10B6F80000234FF0FF3204930793059206938DF8C9
:10B7080053301A93052229786048FFF7A7FA05F104
:10B718000108049B002831D1D90644BF20228DF8A6
:10B7280053201A0744BF2B228DF853202A782A2A3F
:10B738002CD000210A20079AA84698F80030013535
:10B74800303B092B6DD971B326E0514B9C4201D196
:10B75800B468A3E74F4B9C4208BFF4689EE72146B4
:10B768003046FEF7B5F900289ED04FF0FF301DB0E7
:10B77800BDE8F08F252BA7D0A846A0E7434A454649
:10B78800801A0BFA00F018430490BBE7039A111DC6
:10B7980012680391002A01DB079204E0524243F049
:10B7A80002030792049398F800302E2B10D198F8D2
:10B7B800013008F101012A2B37D1039B08F1020857
:10B7C8001A1D1B680392002BB8BF4FF0FF33059377
:10B7D800314D032298F800102846FFF73FFA40B190
:10B7E8004023401B03FA00F0049B08F101080343BF
:10B7F800049398F800100622284808F101078DF8EC
:10B808002810FFF72BFA002834D0254B03BB039BE5
:10B81800073323F0070308330393099B4B44099329
:10B828004CE700FB0232012186E700230A2518466F
:10B838000593884698F800200131303A092A03D93F
:10B84800002BC5D00590C3E705FB00200123F0E7D6
:10B8580003AB00932246134B04A93046FDF7B8FB0F
:10B86800B0F1FF3F8146D8D1A3895B063FF57DAF94
:10B8780009987CE703AB009322460A4B04A930469B
:10B88800FDF756FEECE700BF38BD000874BE00089F
:10B8980058BD000818BD00087ABE00087EBE000822
:10B8A800D98F000861B6000838B50023054C054655
:10B8B80008462360FDF748FA431C02D1236803B108
:10B8C8002B6038BD3019002010B50C46B1F90E10A8
:10B8D80000F0E8F80028ABBF636DA3891B1823F4B8
:10B8E8008053ACBF6365A38110BD2DE9F0411F46AD
:10B8F8008B890546DB050C46164605D50223002232
:10B90800B1F90E1000F068F8A389324623F4805389
:10B91800A381B4F90E103B462846BDE8F04100F07B
:10B9280017B810B50C46B1F90E1000F055F8431CC5
:10B93800A38915BF606523F4805343F48053A38122
:10B9480018BFA38110BDB1F90E1000F013B80000A4
:10B9580038B50546084611460022054C22601A46AD
:10B96800FCF7E8FC431C02D1236803B12B6038BD07
:10B978003019002038B50023054C054608462360D9
:10B98800FDF7FCF9431C02D1236803B12B6038BDD5
:10B998003019002038B50023064C054608461146E4
:10B9A8002360FDF7EEF9431C02D1236803B12B6035
:10B9B80038BD00BF3019002038B50023054C0546B6
:10B9C80008462360FDF7E2F9431C02D1236803B15E
:10B9D8002B6038BD3019002038B505460846114699
:10B9E8000022054C22601A46FDF7D2F9431C02D109
:10B9F800236803B12B6038BD3019002082B001B92B
:10BA080001A942B14BB113780B601278101C18BF12
:10BA1800012002B070471046FBE76FF00100F8E71D
:10BA2800884210B501EB020303D8421E99420CD19B
:10BA380010BD9842F9D28118D21AD34200D110BD54
:10BA480013F8014D01F8014DF7E711F8014B02F821
:10BA5800014FEBE770477047F8B5074614460E46A6
:10BA680021B91146BDE8F840FFF732BC22B9FFF70B
:10BA7800E3FB25462846F8BD00F033F884420FD989
:10BA880021463846FFF724FC05460028F2D0314607
:10BA98002246FDF7F9F931463846FFF7CDFBE9E7CD
:10BAA8003546E7E738B50546084611460022054CF5
:10BAB80022601A46FDF73AF9431C02D1236803B104
:10BAC8002B6038BD3019002049B1FF2A8BBF8A236B
:10BAD8000A700360012088BF4FF0FF3070470846A6
:10BAE800704751F8040C0028A0F10400BCBF0B58A3
:10BAF800C0187047F8B500BFF8BC08BC9E46704730
:0CBB0800F8B500BFF8BC08BC9E467047B2
:10BB180000061016000610164368616E6E656C20EC
:10BB280053657474696E6700707265737320616E13
:10BB38007920427574746F6E00202032387E323856
:10BB48002E352047487A202000202032382E357E96
:10BB580032392047487A2000202032397E32392E67
:10BB6800352047487A2000202032392E357E333060
:10BB78002047487A200020202020322E3447487A57
:10BB880020202020200020202020352E3847487AE9
:10BB980020202020200020204120436820313530FB
:10BBA8004D487A2000202020202530362E3266206D
:10BBB8002020644200202020412043682033304761
:10BBC8000020202041204368616E6E656C20202093
:10BBD800002020202053657474696E67002020209F
:10BBE8004120436820574946492020002020422010
:10BBF8004368203135304D487A20002020204220EB
:10BC080043682033304700202042204368616E6E2D
:10BC1800656C00202042204368205749464920206F
:10BC280000437269746963616C204572726F720DAA
:10BC3800005B4572726F72205D446566616C757455
:10BC480020696E2025732020202020204C494E4555
:10BC5800203A2564200D0A00417474656E5F4F70A8
:10BC680065726174655F4D656D5F525700253032AE
:10BC7800782000434845434B53554D5F4552524F3A
:10BC880052202052656376435243203A20253032B1
:10BC98007820202C20696E6465782025640D0A00C0
:10BCA800576861742048617070656E3F0D00000030
:10BCB8000000000000000102030406070809000054
:10BCC800000001020304000010000020494E460055
:10BCD800696E66004E414E006E616E003000303174
:10BCE80032333435363738394142434445460030DB
:10BCF800313233343536373839616263646566000A
:10BD0800496E66696E697479004E614E00000000E4
:10BD1800000000000000000000000000000000001B
:10BD2800000000000000000000000000000000000B
:10BD380000000000000000000000000000000000FB
:10BD480000000000000000000000000000000000EB
:10BD580000000000000000000000000000000000DB
:10BD680000000000000000000000000000000000CB
:10BD78000080E03779C34143176E05B5B5B89346DF
:10BD8800F5F93FE9034F384D321D30F94877825AAB
:10BD98003CBF737FDD4F1575000000000000F03FC9
:10BDA800000000000000244000000000000059408E
:10BDB8000000000000408F40000000000088C340E1
:10BDC80000000000006AF8400000000080842E4156
:10BDD80000000000D01263410000000084D79741A2
:10BDE8000000000065CDCD41000000205FA00242A8
:10BDF800000000E876483742000000A2941A6D421D
:10BE0800000040E59C30A2420000901EC4BCD6420F
:10BE180000003426F56B0C430080E03779C34143BA
:10BE280000A0D8855734764300C84E676DC1AB4330
:10BE3800003D9160E458E143408CB5781DAF15444E
:10BE480050EFE2D6E41A4B4492D54D06CFF0804429
:10BE5800F64AE1C7022DB544B49DD9794378EA443E
:10BE680005000000190000007D000000232D302B84
:10BE78002000686C4C0065666745464700430050E3
:10BE88004F534958002E0000202020202020202039
:10BE98002028282828282020202020202020202072
:10BEA8002020202020202020881010101010101092
:10BEB80010101010101010100404040404040404DA
:10BEC800040410101010101010414141414141016B
:10BED800010101010101010101010101010101014A
:10BEE8000101011010101010104242424242420259
:10BEF800020202020202020202020202020202021A
:10BF080002020210101010200000000000000000C3
:10BF18000000000000000000000000000000000019
:10BF28000000000000000000000000000000000009
:10BF380000000000000000000000000000000000F9
:10BF480000000000000000000000000000000000E9
:10BF580000000000000000000000000000000000D9
:10BF680000000000000000000000000000000000C9
:10BF780000000000000000000000000000000000B9
:08BF88000000000000000000B1
:08BF9000E04EFF7F01000000FC
:04BF9800AD010008EF
:04BF9C00890100080F
:10BFA00001000000100000000024F4001000002038
:10BFB0000000000038BD000858BD000818BD00088A
:10BFC0000000000000000000000000000000000071
:10BFD0000000000000000000000000000000000061
:10BFE0000000000000000000000000000000000051
:10BFF0000000000000000000000000000000000041
:10C000000000000000000000000000000000000030
:10C0100043000000000000000000000000000000DD
:10C020000000000000000000000000000000000010
:10C0300043000000000000000000000000000000BD
:10C0400000000000000000000000000000000000F0
:10C05000430000000000000000000000000000009D
:10C0600000000000000000000000000000000000D0
:10C07000430000000000000000000000000000007D
:10C0800000000000000000000000000000000000B0
:10C09000430000000000000000000000000000005D
:10C0A0000000000000000000000000000000000090
:10C0B000430000000000000000000000000000003D
:10C0C0000000000000000000000000000000000070
:10C0D000430000000000000000000000000000001D
:10C0E0000000000000000000000000000000000050
:10C0F000D1BA000805BA0008000000008FBE000891
:10C100008DBE00085FBC00085FBC00085FBC000873
:10C110005FBC00085FBC00085FBC00085FBC000893
:10C120005FBC00085FBC0008FFFFFFFFFFFFFFFFD1
:10C13000FFFFFFFFFFFF000001004153434949009B
:10C1400000000000000000000000000000000000EF
:10C150000000000000000000000041534349490076
:10C1600000000000000000000000000000000000CF
:0CC17000000000000000000000000000C3
:0400000508008DE979
:00000001FF
